:1066C800011900000501013C0200000301FA040061
:1066D800FA0500030A0A5A0B001E0C00FA0D000303
:1066E8000E00030F0164100096120132130AFA1407
:1066F800010215000017010A1801FA1905321A01DA
:106708000A1B01FA1C05321FFFFF20FFFF23011E91
:106718002400642A00FA2B00FA2C50782D003D2E14
:1067280000462F001E3000643250783432FA3501AA
:1067380064360164370150380A643C00643E003C0A
:106748003F000140FFFF411450420A5A430AC8441F
:1067580005324500B44600FA47013C4802024C00A5
:10676800FA4EFFFF500C0C510596520A32530B4655
:10677800540A96560202570546580002590A465AC4
:1067880032FA5B010A5C0A325E000A5F00FE61FFB2
:10679800FF64031C6600016701016A0A3C6B000084
:1067A8006C32967300007400007801327901327EF1
:1067B80000FE7FFFFF80FFFF8100008400FE850050
:1067C800AF8600018700FA8901048A000099000059
:1067D8009D0A969E00019FFFFFFAFAFA0065006F76
:1067E80000790083008D009700A100AC00B600C0BE
:1067F80000CA00D400DE00E800F2005B0063006A13
:106808000072007A008200890091009900A100A816
:1068180000B000B800BF00C700CF00D600DF00E618
:1068280000EE00F600400046004C00520059005FA0
:106838000065006B00710077007D00830089008F80
:106848000095009C00A200A800AE00B400BA00C0E9
:1068580000C600CC00D200D900DF00E500EB00F153
:1035E7009007D6E0FEA3E0FF9066CA1269A1E493B4
:1035F700F5999066C8E493FC740193FDEFB5050750
:10360700EEB50403754C009007D61269882275A79A
:103617001085F97185FA727E017F00E57212697A69
:10362700E5712FFF50010E8E588F59900023E0FC53
:10363700A3E0FDEF2DFDEE3CFC8C5A8D5B22E55B94
:10364700F5FBE55AF5FCD29322E55BF5E9E55AF57A
:10365700EAD29422E55BF5EBE55AF5ECD29122E547
:103667005BF5EDE55AF5EED29222E55BF5FDE55AFD
:10367700F5FED28722E55BF5CEE55AF5CFD290224B
:10368700AE58AF5974068E048F05FF12696A8C5ABB
:103697008D5BAE58AF5974068E048F05FF1269957E
:1036A7008C588D59E559455860137406C39559FFD1
:1036B700E49558FE8E588F59785A1269CEE571A84D
:1036C7005AB80015D3955B4010E571C3955BFFE4CD
:1036D700955AFE8E5A8F5B8010E571243CC3955B2B
:1036E700FFE4955AFE8E5A8F5BAE5AAF5B743B6F01
:1036F7004E6006743C6F4E701AAE5AAF5B743B6FE8
:103707004E70057571018003757102755B3A755AC4
:10371700008003757100229000A6E0B40104C20A7C
:103727008002D20A9000A7E0B40104C20B8002D243
:103737000B9000E4E075F0E6A4FFAEF0740A8E0487
:103747008F05FF12696A9007CCECF0A3EDF0A20792
:10375700401674038C068D0712697A7401120039BA
:103767009007CAEEF0A3EFF07E017F009000A2E081
:1037770012697A9000E5E08E048F05FF12696A747A
:103787000AFF12696A8D5E9000EEE075F0E6A4FF0D
:10379700AEF0740A8E048F05FF12696A9007D0ECA9
:1037A700F0A3EDF09000F0E060139000F0E0F5F08A
:1037B700741684FF7E00EF9007DAF0800674649039
:1037C70007DAF09000E6E090008AF0900130E09090
:1037D7000074F09000E8E0900077F0900094E0909B
:1037E7000078F09000DAE0900079F090011AE0900C
:1037F700007DF074E3900089F09000CFE0B40B08EF
:1038070074E3900089F0805A9000CFE0B4191290C9
:1038170000E5E09067CF12008CE493900089F08078
:10382700419000CFE0B41E129000E5E09067ED12E2
:10383700008CE493900089F080289000CFE0B428B2
:10384700129000E5E090681712008CE493900089CD
:10385700F0800F9000CFE0B446089000C6E09000DB
:1038670089F090008DE0FE9000CCE0B5062790002F
:103877008EE0FE9000F8E0B5061B90008FE0FE900A
:1038870000EAE0B5060F900090E0FE90009FE06E22
:1038970070030239FB740490011BF090009FE0B4A1
:1038A7000106740090009FF090009FE0B402067438
:1038B700009000EAF090009FE0B4030674009000C7
:1038C700F7F09000F8E0B4012674009000B3F074AC
:1038D7001C90011EF074009006E0F074009006E161
:1038E700F09000CCE0600674009000CCF08032903D
:1038F70000CCE0601A741C9000B3F0740090011EB5
:10390700F074009006E0F074009006E1F080127405
:103917000090011EF074009000B3F0741C9006E054
:10392700F09000EAE0D39401402774009000B4F0CF
:10393700741B90011DF074009006DCF07400900673
:10394700DDF09000CCE0B4020674019000CCF0806A
:10395700339000CCE0B4021A741B9000B4F07400EA
:1039670090011DF074009006DCF074009006DDF005
:10397700801274009000B4F0740090011DF0741B65
:103987009006DCF09000BFE060147409900122F00B
:1039970074009006E4F074009006E5F0800C740063
:1039A700900122F074099006E4F0D2249000CCE054
:1039B70090008DF09000F8E090008EF09000EAE023
:1039C70090008FF090009FE0900090F090009FE0B3
:1039D700900075F09000BFE0900076F09000F8E05E
:1039E70090007AF09000CCE090007BF09000EAE045
:1039F70090007CF0900091E0FE9000BFE06E603E8A
:103A07009000BFE0600E7409900122F074009006E8
:103A1700E4F0800C7400900122F074099006E4F041
:103A2700900091E060069000BFE07002D224900001
:103A3700BFE0900091F09000BFE0900076F0900119
:103A470002E0B4011790002F740FF0A374FFF090F9
:103A57000031E4F0A3F07402900102F0900102E05B
:103A6700B40341900031E0FEA3E0FF90002FE0FC9B
:103A7700A3E0FD1269C6741012697A74081200393E
:103A8700EF900086F0EF700674FF900086F07400E8
:103A9700900102F0900030E0900087F090002FE056
:103AA700900088F0900093E090004BF090004BE07E
:103AB700240A90004CF090004BE0241490004DF045
:103AC70090004BE0241E90004EF090004BE024281D
:103AD70090004FF090004BE02432900050F090009F
:103AE7004CE0D3943C400B90004CE0C3943C9000D6
:103AF7004CF090004DE0D3943C400B90004DE0C358
:103B0700943C90004DF090004EE0D3943C400B90D5
:103B1700004EE0C3943C90004EF090004FE0D394E9
:103B27003C400B90004FE0C3943C90004FF0900056
:103B370050E0D3943C400B900050E0C3943C90007D
:103B470050F0900057E4F090004BE0643B60079022
:103B5700004BE0B43C2090004BE0B43B067402906D
:103B67000057F090004BE0B43C069000577401F00A
:103B770090004B7401F0900058E4F090004CE06422
:103B87003B600790004CE0B43C2090004CE0B43B15
:103B9700067402900058F090004CE0B43C06900088
:103BA700587401F090004C7401F0900059E4F090C3
:103BB700004DE0643B600790004DE0B43C2090006E
:103BC7004DE0B43B067402900059F090004DE0B40C
:103BD7003C069000597401F090004D7401F090007C
:103BE7005AE4F090004EE0643B600790004EE0B46A
:103BF7003C2090004EE0B43B06740290005AF090CF
:103C0700004EE0B43C0690005A7401F090004E74E8
:103C170001F090005BE4F090004FE0643B60079098
:103C2700004FE0B43C2090004FE0B43B0674029094
:103C3700005BF090004FE0B43C0690005B7401F02D
:103C470090004F7401F090005CE4F0900050E06445
:103C57003B6007900050E0B43C20900050E0B43B3C
:103C670006740290005CF0900050E0B43C069000AF
:103C77005C7401F09000507401F0900093E0FE90A6
:103C870000F6E02E90005EF090005EE0641E600794
:103C970090005EE0B43C0690005EE004F090005EA9
:103CA700E0641D600790005EE0B43B0690005EE0B4
:103CB70014F090005EE0D3943C400B90005EE0C3AC
:103CC700943C90005EF090005EE0D3941E400D900F
:103CD700005EE0C3941E90005FF0800A90005EE0F3
:103CE700241E90005FF0754F1E9000D9E0900051A0
:103CF700F0900051E075F00A84AFF07E00EF4E704F
:103D070006900051E004F0900051E00475F00A8439
:103D1700AFF07E00EF4E7006900051E014F0900077
:103D270051E0B43D069000517401F0900051E02439
:103D37000A900052F0900051E02414900053F09044
:103D47000051E0241E900054F0900051E024289088
:103D57000055F0900051E02432900056F090005248
:103D6700E0D3943C400B900052E0C3943C90005247
:103D7700F0900053E0D3943C400B900053E0C39481
:103D87003C900053F0900054E0D3943C400B9000DB
:103D970054E0C3943C900054F0900055E0D3943C19
:103DA700400B900055E0C3943C900055F0900056AE
:103DB700E0D3943C400B900056E0C3943C900056EF
:103DC700F022C293C294C291C292C287C290E5B553
:103DD70054EFF5B5E5B554DFF5B5C296C295C2A067
:103DE700C297C2A2C2A1E5B554BFF5B5E5B5547FE8
:103DF700F5B5E5B554FBF5B5C20C755C469000DC2E
:103E0700E07005756B028003756B0375530075527F
:103E17000090001874FFF0A374DCF0C212C214C241
:103E270016C218C21AC21C74C8900033F074C89026
:103E37000037F074C890003BF074C890003FF074EE
:103E4700C8900043F074C8900047F0755100755052
:103E570000C207754500E56DB40903756D0075610E
:103E670000900025E4F0A3F0756E10C20FC210C2D7
:103E7700119007CCE0FEA3E0FF740312697A740186
:103E87001200399007CAEEF0A3EFF0C20275550091
:103E970075540090001CE4F0A3F0C2257557007517
:103EA700560090009EE075F032A4FDACF090002D16
:103EB700ECF0A3EDF0C2352275A71085F97185FAEC
:103EC700727E017F00E57212697AE5712FFF50015A
:103ED7000E8E588F59AC5AAD5BEF2DFDEE3CFC8C26
:103EE7005A8D5BD293D294D291D292D287D290E557
:103EF7005BF5FBE55AF5FCE55BF5E9E55AF5EAE51F
:103F07005BF5EBE55AF5ECE55BF5EDE55AF5EEE526
:103F17005BF5FDE55AF5FEE55BF5CEE55AF5CF75A0
:103F2700A7002285F97185FA727E017F00E572127A
:103F3700697AE5712FFF50010E8E588F597E017FE8
:103F470076900117E012697AAC58AD59ED2FFFEC66
:103F57003EFE8E5A8F5BE55BF5E9E55AF5EA900080
:103F67008AE4F07412900061F02285F97185FA7283
:103F77007E017F00E57212697AE5712FFF50010E0D
:103F87008E588F599007CCE0FCA3E0FDEF2DFDEE96
:103F97003CFC8C5A8D5BE55BF5FBE55AF5FC22058D
:103FA7006222A2D8B3400CC296C295C2A0C297C2E1
:103FB700A2C2A1A2D9B340089000E6E090008AF01F
:103FC70075D8402285A77075A710A2D8B34002C242
:103FD70093A2D9B34002C294A2DAB34002C291A21B
:103FE700DBB34002C292A2DCB34002C287A2DDB3B8
:103FF7004002C29075D8408570A722900047E4938D
:104007006406600280FE74C89007D2F8E4F0E8A363
:10401700F075B50075840175A70075FFA090005D68
:10402700E4F075C91075A70F75A1C775A70075D9F5
:104037000075CE0C75A70F75F1FE75F2FF75F307C6
:1040470075F47875A4BA75A5FF75A60775AE0075E2
:10405700AFFF75D48175D5FF75D6FF75D7FF75A7E7
:104067000075A20175A14775F80975D80075D904BF
:1040770075DA0975DB0975D84075A71075D800750D
:10408700D90475DA0975DB0975DC0975DD0975DE93
:104097000975DF0975D84075A70075E60875E7103B
:1040A70075BC0175BE0475BD6C75BE0775BDA07581
:1040B700BE0875BD0175BC0075BB1875BC2075BA07
:1040C7000875E88075D11375A70F75E10575E200CE
:1040D70075C740123DC9759700759780740A1269B4
:1040E7005A7597C0E5975420700280F8758F02754E
:1040F700A700D2AF75980075A90C75A70F75AB43CC
:1041070075ADFB75AC1E75A71075C91875CA007516
:10411700CB0075C80475A700758912758E04758C58
:1041270000758A00C2A9D28C758D00758B00D2AB41
:10413700D28E75EF0675D944C29974C8F50975080A
:10414700001200E375B5001204E374639007D2F818
:10415700E4F0E8A3F012036F74C89007D2F8E4F014
:10416700E8A3F07464F5097508001200E390007580
:10417700E090009FF0C22090009FE0D39403400698
:10418700740090009FF090009FE09062D4F8282878
:10419700738028A2B44002D220802075A70F75F340
:1041A7000F75A700A2A34002D220800F75A70F7535
:0B41B700F31775A700A2A44002D2205D
:0C62D40002419802419A0241A20241B32B
:1041C200A220B34066757108E571D3940E5020E5C4
:1041D200719007D2F8E4F0E8A3F012023E7464F59D
:1041E200097508001200E37871740126F650D9743B
:1041F200029000DBF090009FE0D39403400674002D
:1042020090009FF090009FE09062E0F82828738071
:10421200167400900105F0800E74009000EAF080A0
:074222000674009000F7F0A4
:0C62E00002421102421302421B02422340
:10422900D21F8064757101E571D394075020E5713F
:104239009007D2F8E4F0E8A3F012023E7464F5099D
:104249007508001200E37871740126F650D97401DB
:104259009000DBF090009FE0D39403400674009037
:10426900009FF090009FE09062ECF8282873801678
:104279007400900105F0800E74009000EAF0800649
:0642890074009000F7F044
:0C62EC000242770242790242810242899C
:10428F00C21F900074E0900130F0900075E0900034
:10429F009FF0900076E09000BFF0900077E09000E4
:1042AF00E8F0900078E0900094F0900079E09000B2
:1042BF00DAF090007AE09000F8F090007BE0900048
:1042CF00CCF090007CE09000EAF090007DE090014F
:1042DF001AF09000E5E07006740A9000E5F0900087
:1042EF00C6E0700674E39000C6F09000CCE0049036
:1042FF00008DF09000BFE004900091F012371EE5A2
:10430F00B54401F5B57406900063F0740190006434
:10431F00F07403900066F07405900067F0744D9090
:10432F000068F07406900069F0740090006AF074F1
:10433F000090006FF07400900070F07401900071A5
:10434F00F07400900072F074FF900073F074369068
:10435F000169F0743090016AF0742D90016BF07464
:10436F003290016CF0742090016DF0744D90016EDD
:10437F00F0746590016FF07472900170F074639037
:10438F000171F07420900172F07420900173F07439
:10439F0056900174F07431900175F074329001767B
:1043AF00F07420900177F0900101E0900086F0907A
:1043BF0000B8E0900087F09000B9E0900088F0A27C
:1043CF00B6B39208A2B3B39209A2A4B39222A2A346
:1043DF00B39223900082E4F0756D00743A900792C7
:1043EF00F074FD900793F0900083E4F09007CCE019
:1043FF00FEA3E0FF740312697A740112003990076B
:10440F00CAEEF0A3EFF0756C01900061E4F0C221E9
:10441F00756100C20DD20EC202756F00C227D203A2
:10442F00C228D204C229D205C22412009E755D0093
:10443F00756900755F007563327564007565007589
:10444F006600756700756800900025E4F0A3F075AD
:10445F006A00D2B2D2A4D2B0D2B1D2A3D2A7D2A67E
:10446F00D2A5D2B790009EE0D394FA400674FA908A
:10447F00009EF07E017F00900088E012697A900024
:10448F0087E02FFF50010E90002FEEF0A3EFF0EF1B
:10449F00D394FFEE940F400790002FE4F0A3F09019
:1044AF000086E0700674FF900086F074009000C5DF
:1044BF00F09000DBE0D39402400674019000DBF033
:1044CF009000DCE07005756B028003756B03900044
:1044DF00DDE0D39401400674009000DDF09000E31E
:1044EF00E0C3940A5006740A9000E3F09000EDE0E8
:1044FF00700674019000EDF09000EDE0B4FF0674CB
:10450F00FE9000EDF09000F4E0D394FE400674FEB0
:10451F009000F4F090011AE0D394024006740190D9
:10452F00011AF0900130E0D394014006740190011C
:10453F0030F074019000FAF074019000FBF07400F9
:10454F00900102F0740890011FF07407900120F0A1
:10455F00742A900121F07400900122F074299006C2
:10456F00D8F0D29C9000CDE0D39404400674049010
:10457F0000CDF09000FFE0D3940440067404900047
:10458F00FFF0E56ED394104003756E109006D9E0DE
:10459F00D3940C400674009006D9F09006DDE0D35A
:1045AF00940C400674009006DDF09006E1E0D39481
:1045BF000C400674009006E1F09006E5E0D3940CF1
:1045CF00400674009006E5F0D2EC75CF01A298B3C7
:1045DF004005C298120616E54C6006A299B3B34087
:1045EF00028005C299120AB4E54D64016005E54DDC
:1045FF00B4040280D5C28E7E107F00E56212697A04
:10460F00E58D75F010A4FDACF0EF2DFDEE3CFCE553
:10461F008B75F01084FF7E00ED2FFFEC3EFE8E5267
:10462F008F53D28E9000BFE060099000BFE0C3941B
:10463F003D40028056900027126988900027E0FEC7
:10464F00A3E0FF900029E0FCA3E0FDEFB5053CEEF1
:10465F00B50438B21EA207B34013A21EB34008E53B
:10466F00B54404F5B58006E5B554FBF5B5900029C2
:10467F00E0FEA3E0FF90002BE0FCA3E0FDEF2DFD9B
:10468F00EE3CFC900029ECF0A3EDF09000CCE06044
:10469F00099000CCE0C3940340030247471229C09E
:1046AF00A207B35009900082E0C3942F4002800606
:1046BF009000B6E0F544E54475F005A4FFAEF09028
:1046CF0007D4EEF0A3EFF09000A3E0C3955F40078F
:1046DF00E55DC3955E50079007D4E4F0A3F0AE2DCF
:1046EF00AF2E9007D4E0FCA3E0FDEFD39DEE9C40EE
:1046FF0020E5B5547FF5B59000CCE0B402099000E9
:10470F00EAE0C3940240028006E5B54440F5B58067
:10471F0027900082E0C394465006E5B54480F5B576
:10472F009000CCE0B402099000EAE0C3940240028A
:10473F008006E5B554BFF5B59000CCE0B403241264
:10474F002ADBAE2DAF2E9007D4E0FCA3E0FDEFD314
:10475F009DEE9C4008E5B54480F5B58006E5B5545F
:10476F007FF5B5A2B6300801B35003024D87A2B64C
:10477F00300801B35003024D87A2B6300A01B3507F
:10478F0003024C12756C009000BFE0B43D1975E741
:10479F0000A20AB34008E5B554FBF5B58006E5B5B0
:1047AF004404F5B575E710055CA20CB3B35013AE16
:1047BF0052AF53900018E0FCA3E0FDEDC39FEC9EB9
:1047CF0040030248EFE56BB4032EA225B34022E568
:1047DF005CB43B03756B01E55CC3943B50069000E2
:1047EF00617401F0E55CD3943B4006740290006164
:1047FF00F0755C01D2258062E56BB40206756B0122
:10480F00755C3BE55CB43B05755C01804D900061C8
:10481F00E07038E55CC3943B50069000617401F082
:10482F00E55CD3943B40067402900061F0E55CC3F5
:10483F00943B5002D221E55CD3943B4002D221C27B
:10484F0096C295C2A0C297C2A2C2A19000DCE0B4EA
:10485F000105123DC98003755C01AE54AF55AC52D2
:10486F00AD53EF2DFDEE3CFC74028C068D0712004C
:10487F00398E548F559000BFE060099000BFE0C3A0
:10488F00943D40028043900027E0FEA3E0FF90009C
:10489F00BFE08E048F05FF12696A74018C068D07C5
:1048AF0012003990002BEEF0A3EFF090002BE0F800
:1048BF00A3E0900029C8F0A3C8F0900027E4F0A36C
:1048CF00F0C21EE5B554FBF5B5A2A4B34002C22257
:1048DF00A2A3B34002C223A221B34002C221803A55
:1048EF00AE54AF55AC52AD53EF2DFDEE3CFC740101
:1048FF008C068D071200398E548F55E56BC39402C9
:10490F00500DAC52AD5374B8C39D740B9C400280D4
:10491F0009123DC97406900061F0E55CB43B127456
:10492F0003900061F0D2219000DCE0B40103123D4E
:10493F00C9AE56AF57AC52AD53EF2DFDEE3CFC8CCC
:10494F00568D57AE52AF53EFD39DEE9C4011900052
:10495F001FE0FAA3E0FBEBC394E8EA940340028064
:10496F000690001F12698890001CE0FEA3E0FFACC8
:10497F0052AD53EF2DFDEE3CFC90001CECF0A3ED7F
:10498F00F09000DCE0B40118AE52AF537405126919
:10499F007A7401120039900018EEF0A3EFF0801135
:1049AF00AE52AF53740212697A900018EEF0A3EF73
:1049BF00F0C28E758D00758B007562007553017591
:1049CF005200D28EE55C240E75F00F84AFF07E009E
:1049DF00EF4E707590001CE0F8A3E090001AC8F03D
:1049EF00A3C8F090001AE0FEA3E0FFEF4E600B7C2F
:1049FF007F7DC41268688E508F5190001CE4F0A325
:104A0F00F0AE50AF517428BE00039F5010E5612FD8
:104A1F00FF50010E74011200398E508F5185516174
:104A2F009000E3E0A850B8000DD395514008E55130
:104A3F00900060F080099000E3E014900060F0E5D2
:104A4F006B6006755100755000E55C640B6005E501
:104A5F005CB429099000CCE0600312202B90005E1B
:104A6F00E0655C600790005FE0B55C03756D00A2C8
:104A7F000DB35006A20CB3B34003024B3190009814
:104A8F00E0B4017390011AE0B40214120C559000B7
:104A9F008BE075F0BEA4FFAEF08E5A8F5B8056E5AB
:104AAF006575F00A84FF7E009005921269A1E0F50A
:104ABF0059755800AE58AF599000BDE012697A741D
:104ACF00648E048F05FF12696A8C5A8D5BE55B90CB
:104ADF00001EF0AE58AF59900096E012697A7464D8
:104AEF008E048F05FF12696A74BE8C068D071269DA
:104AFF007A8E5A8F5B8017900096E075F0BEA4FFF8
:104B0F00AEF08E5A8F5B9000BDE090001EF0E55F17
:104B1F00C394CC5006900096E070028003123EBF03
:104B2F00D20DE56BB40106E55C6411600280097576
:104B3F006E019000627401F0E56B6003024C0D9002
:104B4F0000DFE0600D90008AE0A850B80006955194
:104B5F00400280409000DFE0B4021F90004BE06500
:104B6F005C600F90004CE0655C600790004DE0B515
:104B7F005C03756E03756A00800CC200756A009045
:104B8F000025E4F0A3F090008AE06006740990001D
:104B9F0061F0806A90004BE0B55C0B756E01900080
:104BAF00627401F0805890004CE0B55C0B756E019B
:104BBF007402900062F0804690004DE0B55C0B757A
:104BCF006E017403900062F0803490004EE0B55C8B
:104BDF000B756E017404900062F0802290004FE01C
:104BEF00B55C0B756E017405900062F0801090003B
:104BFF0050E0B55C09756E017406900062F0A20A70
:104C0F00B39208A20AB330B601B35003024D8775B1
:104C1F006C019000BFE0B43D1975E700A20AB340E4
:104C2F0008E5B54404F5B58006E5B554FBF5B57553
:104C3F00E710E5B54401F5B5742F900082F0A20A94
:104C4F009208E55CD3944A4014D20CE55CD394856A
:104C5F00400B7404900061F0D221755C469000E720
:104C6F00E0B40107E568C3941440028009123DC9FE
:104C7F007413900061F0A227300301B35017A227DD
:104C8F00B34008E5B54408F5B58006E5B554F7F52A
:104C9F00B5A2279203A228300401B35017A228B35C
:104CAF004008E5B54440F5B58006E5B554BFF5B508
:104CBF00A2289204A229300501B35017A229B340AC
:104CCF0008E5B54480F5B58006E5B5547FF5B5A286
:104CDF00299205A22A300601B35017A22AB3400821
:104CEF00E5B54404F5B58006E5B554FBF5B5A22A44
:104CFF009206900115E0A850B80005D39551500DBC
:104D0F00900114E0A850B80004955150028008E5B6
:104D1F00B54402F5B58017900116E0D3955F4008B2
:104D2F00E5B54402F5B58006E5B554FDF5B5E56882
:104D3F00C394415009740E900061F0123DC9900068
:104D4F0069E0FE900065E0C39E4009900065E0D3E6
:104D5F009406400974FB900061F0123DC990006EFB
:104D6F00E0601590006EE0FE900068E06E600974E0
:104D7F00FE900061F0123DC9A221B3400CC296C251
:104D8F0095C2A0C297C2A2C2A1900117E0600CAE5B
:104D9F0050AF517414BE00059F4002803790009FA2
:104DAF00E09062F8F8282873802A8028A2A3B350D5
:104DBF0005A223B340028005123F2AD2238015A2F9
:104DCF00A4B35005A222B340028005123F2AD2227B
:044DDF0080028000CE
:1062F800024DB7024DB9024DBB024DCE024DE1022F
:026308004DE363
:104DE300A20FB3B35008900051E0655C60028036B7
:104DF300A201B35006A200B3B340028023123615BA
:104E03001236459000F8E0B40113A202B34008E55E
:104E1300B54480F5B58006E5B5547FF5B575A700B3
:104E2300C20FD210D211A210B3B35008900052E0B7
:104E3300655C60028036A201B35006A200B3B340A2
:104E43000280231236151236509000F8E0B4011395
:104E5300A202B34008E5B54480F5B58006E5B55434
:104E63007FF5B575A700D20FC210D211A211B3B34B
:104E73005008900053E0655C60028036A201B35095
:104E830006A200B3B34002802312361512365B909C
:104E930000F8E0B40113A202B34008E5B54480F57D
:104EA300B58006E5B5547FF5B575A700D20FD210CE
:104EB300C211A20FB3B35008900054E0655C6002C6
:104EC3008036A201B35006A200B3B340028023127E
:104ED30036151236669000F8E0B40113A202B3400F
:104EE30008E5B54480F5B58006E5B5547FF5B5759D
:104EF300A700C20FD210D211A210B3B35008900072
:104F030055E0655C60028036A201B35006A200B38F
:104F1300B3400280231236151236719000F8E0B4C4
:104F23000113A202B34008E5B54480F5B58006E558
:104F3300B5547FF5B575A700D20FC210D211A211D7
:104F4300B3B35008900056E0655C60028036A2015E
:104F5300B35006A200B3B3400280231236151236B3
:104F63007C9000F8E0B40113A202B34008E5B54415
:104F730080F5B58006E5B5547FF5B575A700D20F6A
:104F8300D210C211E56E90630AF82828730256A165
:044F93009000FFE0AB
:06630A00024F90024F93C8
:104F970090633DF8282873121B078012121B0780A5
:0E4FA7000D121B918008121C3D8003121C3D50
:0F633D00024F9E024FA3024FA8024FAD024FB274
:104FB500756E020256A1121D69121E80A235B340FC
:104FC500229000C1E0F56A900092E0256AFE90000B
:104FD50060E075F01E84FC7F00EE2CF533741090B4
:104FE5000061F09007CAE0FEA3E0FF740A12697A37
:104FF50090001AE0FCA3E0FD74098F02FF12696AB4
:105005008D078C038E048A058B061268689007CE7F
:10501500EEF0A3EFF074F0BE00039F500B74F09018
:1050250007CEF8E4F0E8A3F0E5337003753301909B
:1050350007CEE0FEA3E0FFE5332FFF50010E9007FA
:0D504500CEEEF0A3EFF0756E03900062E078
:03631000024FBB7E
:1050520090634CF82828738034A2364003756E0A98
:10506200802BA2364003756E0B8022A23640037558
:105072006E0C8019A2364003756E0D8010A2364068
:0D50820003756E0E8007A2364003756E0F99
:10634C0002505902505B02506402506D02507602AA
:05635C00507F02508893
:10508F000256A19006D9E06003122114900118E096
:10509F00B40114900119E0A850B8000495515007BD
:1050AF00E55DC3955E4002800302513C9000CDE068
:1050BF00D39402403F9000A1E02403A850B800040D
:1050CF00955150099000A3E0D3955F50028008D20C
:1050DF00017408900061F09000A1E0A850B800059D
:1050EF00D39551500B9000A3E02403C3955F50025A
:1050FF00C20180399000A1E02403A850B8000495A4
:10510F00515007E55DC3955E40028008D2017408D7
:10511F00900061F09000A1E0A850B80005D3955120
:10512F005009E55E240FC3955D5002C2019000E760
:10513F00E07007E568C3941440028002D201A20117
:10514F004005756E04800A756E10900025E4F0A37B
:10515F00F0A207B34029E56575F00A84FF7E009041
:10516F0005921269A1E0C394695005122060800F67
:10517F009007CCE0F8A3E09007CAC8F0A3C8F002EC
:06518F0056A19000CDE0E6
:06631300025092025191BC
:10519500906361F8282873120D3F8012120D3F802D
:0E51A5000D120EED8008120F9F8003120F9F57
:0F63610002519C0251A10251A60251AB0251B050
:1051B3009006DDE060031221F0756E050256A11220
:1051C30010AB756E069006E1E060031222E0025612
:1051D300A190001EE06006A207B3B34002801D90B9
:1051E300001EE02528FFAE2750010E8E278F28E5ED
:1051F3005CD3940A500690001EE014F01212F1756D
:105203006E079006E5E060031223BC0256A19001ED
:105213001AE0B40203120CCD12154E756E08025635
:10522300A112190AA20FB35005A210B340028006BF
:10523300D20FD210D211756E100256A10256A19050
:105243000035E0C394465008C2967446900035F08A
:10525300900057E0B4011DE5332406F5339007CEE3
:10526300E0FEA3E0FF74062FFF50010E9007CEEE81
:10527300F0A3EFF0900057E0B4021DE533240CF5E2
:10528300339007CEE0FEA3E0FF740C2FFF50010E16
:105293009007CEEEF0A3EFF08533597558009000D8
:1052A3004BE0F571123687E55B900035F090000C0A
:1052B300E558F0A3E559F0E571900036F0C213907C
:1052C30007CEE0F558A3E0F55990004BE0F57112D5
:1052D3003687E55B900033F0900000E558F0A3E5D6
:1052E30059F0E571900034F0C212E56BB401057515
:1052F3006E0B8003756E030256A1900039E0C394D0
:10530300465008C2957446900039F0900058E0B4B6
:10531300011DE5332406F5339007CEE0FEA3E0FF3D
:1053230074062FFF50010E9007CEEEF0A3EFF0901E
:105333000058E0B4021DE533240CF5339007CEE0AA
:10534300FEA3E0FF740C2FFF50010E9007CEEEF08A
:10535300A3EFF085335975580090004CE0F57112B6
:105363003687E55B900039F090000EE558F0A3E531
:1053730059F0E57190003AF0C2159007CEE0F55868
:10538300A3E0F55990004CE0F571123687E55B9088
:105393000037F0900002E558F0A3E559F0E571906D
:1053A3000038F0C214E56BB40105756E0C8003750B
:1053B3006E030256A190003DE0C394465008C2A07C
:1053C300744690003DF0900059E0B4011DE533248C
:1053D30006F5339007CEE0FEA3E0FF74062FFF50DF
:1053E300010E9007CEEEF0A3EFF0900059E0B40267
:1053F3001DE533240CF5339007CEE0FEA3E0FF74E4
:105403000C2FFF50010E9007CEEEF0A3EFF0853383
:105413005975580090004DE0F571123687E55B90A1
:10542300003DF0900010E558F0A3E559F0E57190C8
:10543300003EF0C2179007CEE0F558A3E0F559906F
:10544300004DE0F571123687E55B90003BF090006C
:1054530004E558F0A3E559F0E57190003CF0C2165D
:10546300E56BB40105756E0D8003756E030256A1DD
:10547300900041E0C394465008C29774469000419F
:10548300F090005AE0B4011DE5332406F53390078C
:10549300CEE0FEA3E0FF74062FFF50010E9007CE6F
:1054A300EEF0A3EFF090005AE0B4021DE533240CB4
:1054B300F5339007CEE0FEA3E0FF740C2FFF5001FD
:1054C3000E9007CEEEF0A3EFF08533597558009098
:1054D300004EE0F571123687E55B900041F09000D5
:1054E30012E558F0A3E559F0E571900042F0C219B6
:1054F3009007CEE0F558A3E0F55990004EE0F57122
:10550300123687E55B90003FF0900006E558F0A364
:10551300E559F0E571900040F0C218E56BB4010560
:10552300756E0E8003756E030256A1900045E0C3AD
:1055330094465008C2A27446900045F090005BE088
:10554300B4011DE5332406F5339007CEE0FEA3E056
:10555300FF74062FFF50010E9007CEEEF0A3EFF07D
:1055630090005BE0B4021DE533240CF5339007CEC5
:10557300E0FEA3E0FF740C2FFF50010E9007CEEE68
:10558300F0A3EFF085335975580090004FE0F571A3
:10559300123687E55B900045F0900014E558F0A3C0
:1055A300E559F0E571900046F0C21B9007CEE0F597
:1055B30058A3E0F55990004FE0F571123687E55B8B
:1055C300900043F0900008E558F0A3E559F0E57129
:1055D300900044F0C21AE56BB40105756E0F8003A9
:1055E300756E030256A1900049E0C394465008C269
:1055F300A17446900049F090005CE0B4011DE533CE
:105603002406F5339007CEE0FEA3E0FF74062FFFD8
:1056130050010E9007CEEEF0A3EFF090005CE0B4E3
:10562300021DE533240CF5339007CEE0FEA3E0FF23
:10563300740C2FFF50010E9007CEEEF0A3EFF08510
:105643003359755800900050E0F571123687E55BC9
:10565300900049F0900016E558F0A3E559F0E57184
:1056630090004AF0C21D9007CEE0F558A3E0F5592B
:10567300900050E0F571123687E55B900047F0909B
:10568300000AE558F0A3E559F0E571900048F0C22F
:0E5693001CE56BB40103756B00756E0380009F
:106319000251C20251D402521102522402523F02C6
:1063290052420252FD0253B802547302552E0255CD
:04633900E90256A17E
:1056A100900033E0B55C028003025743A2124072BE
:1056B100900000E0FEA3E0FFEF4E6021AE54AF5535
:1056C100900000E0FCA3E0FD12000374068E048F3D
:1056D10005FF12696A900000ECF0A3EDF090003430
:1056E100E0601A900000E0FEA3E0FFAC54AD55EF7E
:1056F1002DFDEE3CFC900000ECF0A3EDF0900034A9
:10570100E0D39401401A900000E0FEA3E0FFAC5406
:10571100AD55EF2DFDEE3CFC900000ECF0A3EDF05B
:10572100D212AE52AF53900000E0FCA3E0FDEFC3F4
:105731009DEE9C400D123F71D296C21274C890002A
:1057410033F0A212B3B35007900033E0B55C02808E
:105751000D123F71D29674C8900033F0C2129000BE
:1057610035E0B55C0280030257FEA213407290003F
:105771000CE0FEA3E0FFEF4E6021AE54AF55900068
:105781000CE0FCA3E0FD12000374068E048F05FFFC
:1057910012696A90000CECF0A3EDF0900036E06025
:1057A1001A90000CE0FEA3E0FFAC54AD55EF2DFDC7
:1057B100EE3CFC90000CECF0A3EDF0900036E0D351
:1057C1009401401A90000CE0FEA3E0FFAC54AD55EB
:1057D100EF2DFDEE3CFC90000CECF0A3EDF0D213AC
:1057E100AE52AF5390000CE0FCA3E0FDEFC39DEE81
:1057F1009C400AC2967446900035F0C213A213B3BE
:10580100B35007900035E0B55C02800AC296744639
:10581100900035F0C213900037E0B55C02800302BE
:1058210058B9A2144072900002E0FEA3E0FFEF4ECF
:105831006021AE54AF55900002E0FCA3E0FD1200E0
:105841000374068E048F05FF12696A900002ECF062
:10585100A3EDF0900038E0601A900002E0FEA3E0B2
:10586100FFAC54AD55EF2DFDEE3CFC900002ECF089
:10587100A3EDF0900038E0D39401401A900002E0CB
:10588100FEA3E0FFAC54AD55EF2DFDEE3CFC9000C6
:1058910002ECF0A3EDF0D214AE52AF53900002E04F
:1058A100FCA3E0FDEFC39DEE9C400D123F71D2952C
:1058B100C21474C8900037F0A214B3B3500790001B
:1058C10037E0B55C02800D123F71D29574C890002B
:1058D10037F0C214900039E0B55C028003025974BC
:1058E100A215407290000EE0FEA3E0FFEF4E602192
:1058F100AE54AF5590000EE0FCA3E0FD120003741E
:10590100068E048F05FF12696A90000EECF0A3ED7C
:10591100F090003AE0601A90000EE0FEA3E0FFACC8
:1059210054AD55EF2DFDEE3CFC90000EECF0A3EDD7
:10593100F090003AE0D39401401A90000EE0FEA3EB
:10594100E0FFAC54AD55EF2DFDEE3CFC90000EECAC
:10595100F0A3EDF0D215AE52AF5390000EE0FCA3D0
:10596100E0FDEFC39DEE9C400AC29574469000395C
:10597100F0C215A215B3B35007900039E0B55C022F
:10598100800AC2957446900039F0C21590003BE040
:10599100B55C028003025A2FA2164072900004E007
:1059A100FEA3E0FFEF4E6021AE54AF55900004E03E
:1059B100FCA3E0FD12000374068E048F05FF12693B
:1059C1006A900004ECF0A3EDF090003CE0601A90C6
:1059D1000004E0FEA3E0FFAC54AD55EF2DFDEE3C1D
:1059E100FC900004ECF0A3EDF090003CE0D39401B6
:1059F100401A900004E0FEA3E0FFAC54AD55EF2D3A
:105A0100FDEE3CFC900004ECF0A3EDF0D216AE529A
:105A1100AF53900004E0FCA3E0FDEFC39DEE9C407A
:105A21000D123F71D2A0C21674C890003BF0A216AD
:105A3100B3B3500790003BE0B55C02800D123F719B
:105A4100D2A074C890003BF0C21690003DE0B55C56
:105A5100028003025AEAA2174072900010E0FEA3EE
:105A6100E0FFEF4E6021AE54AF55900010E0FCA373
:105A7100E0FD12000374068E048F05FF12696A901F
:105A81000010ECF0A3EDF090003EE0601A900010E1
:105A9100E0FEA3E0FFAC54AD55EF2DFDEE3CFC90D4
:105AA1000010ECF0A3EDF090003EE0D39401401A19
:105AB100900010E0FEA3E0FFAC54AD55EF2DFDEEDC
:105AC1003CFC900010ECF0A3EDF0D217AE52AF53B6
:105AD100900010E0FCA3E0FDEFC39DEE9C400AC2E4
:105AE100A0744690003DF0C217A217B3B3500790BF
:105AF100003DE0B55C02800AC2A0744690003DF012
:105B0100C21790003FE0B55C028003025BA5A218BA
:105B11004072900006E0FEA3E0FFEF4E6021AE541C
:105B2100AF55900006E0FCA3E0FD12000374068E61
:105B3100048F05FF12696A900006ECF0A3EDF09066
:105B41000040E0601A900006E0FEA3E0FFAC54AD17
:105B510055EF2DFDEE3CFC900006ECF0A3EDF0902E
:105B61000040E0D39401401A900006E0FEA3E0FF5C
:105B7100AC54AD55EF2DFDEE3CFC900006ECF0A3CE
:105B8100EDF0D218AE52AF53900006E0FCA3E0FD59
:105B9100EFC39DEE9C400D123F71D297C21874C89D
:105BA10090003FF0A218B3B3500790003FE0B55CFE
:105BB10002800D123F71D29774C890003FF0C21855
:105BC100900041E0B55C028003025C60A219407262
:105BD100900012E0FEA3E0FFEF4E6021AE54AF55FE
:105BE100900012E0FCA3E0FD12000374068E048F06
:105BF10005FF12696A900012ECF0A3EDF0900042EB
:105C0100E0601A900012E0FEA3E0FFAC54AD55EF46
:105C11002DFDEE3CFC900012ECF0A3EDF090004263
:105C2100E0D39401401A900012E0FEA3E0FFAC54CF
:105C3100AD55EF2DFDEE3CFC900012ECF0A3EDF024
:105C4100D219AE52AF53900012E0FCA3E0FDEFC3B6
:105C51009DEE9C400AC2977446900041F0C219A281
:105C610019B3B35007900041E0B55C02800AC297B6
:105C71007446900041F0C219900043E0B55C028087
:105C810003025D1BA21A4072900008E0FEA3E0FF30
:105C9100EF4E6021AE54AF55900008E0FCA3E0FD4B
:105CA10012000374068E048F05FF12696A900008C2
:105CB100ECF0A3EDF0900044E0601A900008E0FEE3
:105CC100A3E0FFAC54AD55EF2DFDEE3CFC90000878
:105CD100ECF0A3EDF0900044E0D39401401A900061
:105CE10008E0FEA3E0FFAC54AD55EF2DFDEE3CFC0A
:105CF100900008ECF0A3EDF0D21AAE52AF53900031
:105D010008E0FCA3E0FDEFC39DEE9C400D123F7146
:105D1100D2A2C21A74C8900043F0A21AB3B35007BA
:105D2100900043E0B55C02800D123F71D2A274C8AD
:105D3100900043F0C21A900045E0B55C0280030276
:105D41005DD6A21B4072900014E0FEA3E0FFEF4E6F
:105D51006021AE54AF55900014E0FCA3E0FD1200A9
:105D61000374068E048F05FF12696A900014ECF02B
:105D7100A3EDF0900046E0601A900014E0FEA3E06D
:105D8100FFAC54AD55EF2DFDEE3CFC900014ECF052
:105D9100A3EDF0900046E0D39401401A900014E086
:105DA100FEA3E0FFAC54AD55EF2DFDEE3CFC9000A1
:105DB10014ECF0A3EDF0D21BAE52AF53900014E0FF
:105DC100FCA3E0FDEFC39DEE9C400AC2A274469085
:105DD1000045F0C21BA21BB3B35007900045E0B5CC
:105DE1005C02800AC2A27446900045F0C21B90007A
:105DF10047E0B55C028003025E91A21C40729000F4
:105E01000AE0FEA3E0FFEF4E6021AE54AF559000D3
:105E11000AE0FCA3E0FD12000374068E048F05FF67
:105E210012696A90000AECF0A3EDF0900048E0607E
:105E31001A90000AE0FEA3E0FFAC54AD55EF2DFD32
:105E4100EE3CFC90000AECF0A3EDF0900048E0D3AA
:105E51009401401A90000AE0FEA3E0FFAC54AD5556
:105E6100EF2DFDEE3CFC90000AECF0A3EDF0D21C0E
:105E7100AE52AF5390000AE0FCA3E0FDEFC39DEEEC
:105E81009C400D123F71D2A1C21C74C8900047F012
:105E9100A21CB3B35007900047E0B55C02800D121D
:105EA1003F71D2A174C8900047F0C21C900049E034
:105EB100B55C028003025F4CA21D4072900016E0A7
:105EC100FEA3E0FFEF4E6021AE54AF55900016E007
:105ED100FCA3E0FD12000374068E048F05FF126916
:105EE1006A900016ECF0A3EDF090004AE0601A9081
:105EF1000016E0FEA3E0FFAC54AD55EF2DFDEE3CE6
:105F0100FC900016ECF0A3EDF090004AE0D3940170
:105F1100401A900016E0FEA3E0FFAC54AD55EF2D02
:105F2100FDEE3CFC900016ECF0A3EDF0D21DAE525C
:105F3100AF53900016E0FCA3E0FDEFC39DEE9C4043
:105F41000AC2A17446900049F0C21DA21DB3B3500C
:105F510007900049E0B55C02800AC2A17446900036
:105F610049F0C21D9000EAE0B40202800302609091
:105F7100900084E0D395645064900084E0F404259B
:105F810064FE9000EDE08E00F5F0E884FF7E008F66
:105F910071EFC39410500CEF8571F0A4FDACF08D3E
:105FA1007180037571FF900084E0D39571400B906F
:105FB1000084E0C39571F56F8003756F009001084F
:105FC100E0D3956F4006900108E0F56F900109E07C
:105FD100C3956F5006900109E0F56F8071900084C0
:105FE100E0C39564FE9000EDE08E00F5F0E884FFDB
:105FF1007E008F71EFC39410500CEF8571F0A4FDFA
:10600100ACF08D7180037571FF85715975580090E1
:106011000084E02559FFAE5850010E8E588F5974F7
:10602100FFBE0009D39F400585596F8003756FFF3F
:10603100900108E0D3956F4006900108E0F56F905C
:106041000109E0C3956F5006900109E0F56FA207C1
:10605100B3B3500D900085E0FE9000F5E0D39E5063
:1060610002800E7407900061F0E5B5547FF5B580AC
:106071001B75A710E5CDC3956F4008E5B554BFF575
:10608100B58006E5B54440F5B575A70075A7009044
:10609100010FE0A850B80005D39551501690010E9C
:1060A100E0A850B8000D95514009900110E0D3953A
:1060B1005F4002803175A710E55145506007E5CD7D
:1060C100C394BF4002800EE5B54420F5B5E5B54463
:1060D10010F5B5800CE5B554DFF5B5E5B554EFF530
:1060E100B575A700802F75A710E55145506007E5EC
:1060F100CDC394404002800EE5B54420F5B5E5B529
:106101004410F5B5800CE5B554DFF5B5E5B554EFB0
:10611100F5B575A700E56DC39409500AA2EDB3402A
:1061210005C2ED122C7AAE52AF537410C39F74277F
:106131009E400C900083E0C3945A40030262D1A2B6
:106141000CB34009123DC97406900061F0A220B35E
:106151004008E5B54404F5B58006E5B554FBF5B551
:10616100900083E0D394014013A20EB3500EE55F7B
:10617100D394334007E55FC394CC4002802FE5B54B
:106181004401F5B5742F900082F0900096E075F00F
:10619100BEA4FFAEF08E5A8F5B7402BE000AD39F7D
:1061A1004006755B02755A00123EBFD20E90008305
:1061B100E0D394014007E55FC3941A40028002C214
:1061C1000E9006D9E06003122114A227300301B317
:1061D1005017A227B34008E5B54408F5B58006E598
:1061E100B554F7F5B5A22792039006DDE0600312DE
:1061F10021F0A228300401B35017A228B34008E5CA
:10620100B54440F5B58006E5B554BFF5B5A2289271
:10621100049006E1E060031222E0A229300501B3F7
:106221005017A229B34008E5B54480F5B58006E5CD
:10623100B5547FF5B5A22992059006E5E0600312F9
:1062410023BCA22A300601B35017A22AB34008E5A5
:10625100B54404F5B58006E5B554FBF5B5A22A921F
:1062610006900083E0C3945A5010E56DB40909907B
:106271000083E004F0756D00803BE56DB4090375A2
:106281006D00755300755200758D00758B00756238
:1062910000900082E0C394465008900082E004F030
:1062A10080067446900082F0900082E0B44606E5D4
:1062B100B554FEF5B5900083E0D394014007E5683D
:1062C100C3944140028009740E900061F0123DC9EF
:0362D1000245D9AA
:106370000000010001400160018001A001C001E0B6
:1063800002000300039603B603D603F404000500DD
:106390000512052405360548055A056C057E05904D
:1063A00005A805C005DE0600061406280646066E8A
:1063B00006AE00FF013F015F017F019F01BF01DFCA
:1063C00001FF02FF039503B503D503F303FF04FFA9
:1063D00005110523053505470559056B057D058F15
:1063E00005A705BF05DD05F1061306270645066D61
:1063F00006AD06ED0FAA0FA50F9F0F9A0F940F8DF4
:106400000F870F800F780F710F680F600F570F4EB7
:106410000F450F3B0F300F250F1A0F0E0F020EF511
:106420000EE80EDB0ECC0EBE0EAE0E9F0E8E0E7D57
:106430000E6C0E5A0E470E340E200E0C0DF70DE2A8
:106440000DCB0DB50D9D0D850D6D0D540D3A0D2027
:106450000D050CE90CCE0CB10C940C760C580C3AD2
:106460000C1B0BFB0BDB0BBB0B9A0B790B570B3588
:106470000B130AF10ACE0AAB0A870A640A400A1C07
:1064800009F809D409B0098C09670943091F08FBF9
:1064900008D608B2088E086A0846082307FF07DCFA
:1064A00007B9079607730751072F070D06EC06CAB1
:1064B00006AA068906690649062A060A05EC05CDDC
:1064C00005B0059205750558053C0520050504EA4B
:1064D00004CF04B5049C04820469045104390422E5
:1064E000040B03F403DE03C803B2039D03890375A1
:1064F0000361034D033B03280316030402F202E188
:1065000002D102C002B002A00291028202730265AF
:1065100002570249023C022F02220216020901FD23
:1065200001F201E601DB01D001C601BB01B101A707
:10653000019D0194018B0182017901700168016064
:10654000015801500148014101390132012B012557
:10655000011E01180111010B010500FF00FA0FA631
:106560000FA00F990F920F8B0F840F7C0F740F6B7E
:106570000F620F580F4E0F430F380F2C0F1F0F12C3
:106580000F050EF70EE80ED80EC80EB70EA50E9327
:106590000E800E6C0E580E420E2C0E150DFD0DE4E5
:1065A0000DCB0DB10D950D790D5D0D3F0D200D013C
:1065B0000CE10CC00C9E0C7C0C590C350C100BEA39
:1065C0000BC40B9E0B760B4F0B260AFD0AD40AAAAE
:1065D0000A800A550A2A09FF09D409A8097C09502A
:1065E000092508F908CD08A10875084A081E07F30F
:1065F00007C8079D07730749072006F706CE06A6BA
:10660000067E06570630060A05E405BF059B05779A
:1066100005540532051004EF04CE04AE048F047156
:1066200004530435041903FD03E203C703AD0394C7
:10663000037B0363034B0334031E030802F302DEF0
:1066400002CA02B602A30291027F026D025C024CF2
:10665000023C022C021D020E020001F201E401D7ED
:1066600001CA01BE01B101A6019A018F0185017A1B
:1066700001700166015D0153014A01410139013197
:106680000129012101190112010B010400FD00F78C
:1066900000F000EA00E400DE00D900D300CE00C91B
:1066A00000C400BF00BA00B500B100AD00A800A44E
:1066B00000A0009C009900950091008E008A008740
:0866C00000840081007E007BD4
:10009E007546009007D6E4F0A3F0753000752F007A
:1000AE00754C00754D00C232D23374FE9007E0F8E5
:1000BE00E4F0E8A3F074FE9007E2F8E4F0E8A3F0B1
:1000CE00745A9007E4F0745A9007E5F0D234C226C1
:1000DE00C236C23122750B00750A00AE0AAF0BACE8
:1000EE0008AD09EDC39FEC9E401674FF12695A7558
:1000FE00CF01780B740126F6500418E436F650DB67
:10010E002290005DE0B4AA1C900792E0B43C1590DA
:10011E0007D2E0FEA3E0FFEF4E6009741EBE00049E
:10012E00D39F500302023D755B00755A0075F809A6
:10013E009007D2E0FEA3E0FF74076F4E6006740EC8
:10014E006F4E7006743A900792F09007D2E0FEA3BD
:10015E00E0FF7408BE001ED39F401A7E017F0890F8
:10016E0007D2E0FCA3E0FD1DBDFF011C1200038EB3
:10017E00588F59801F9007D2E0FEA3E0FF7408123B
:10018E0069BE8F048E057E017F08CDCCCD12000393
:10019E008E588F59AE5AAF5B740CD39F74019E501C
:1001AE0003020238A2F9B3407EE55B455A7003752F
:1001BE00A382AE5AAF5B74016F4E700375A300AE8F
:1001CE005AAF5B74026F4E700D9007D3E075F0025C
:1001DE00A4FDACF08DA3AE5AAF5B74036F4E7003EB
:1001EE0075A300AE5AAF5B7403BE00039F5013ACF1
:1001FE0058AD59ED2FFFEC3EFE90008E1269A1E036
:10020E00F5A3AE5AAF5BEFB40B09EEB4010574144F
:10021E0012695AAE5AAF5BEFB40B07EEB401037519
:10022E00F80D785A1269CE0201A290005DE4F02218
:10023E00755B00755A0075F8099007D2E0FEA3E0D1
:10024E00FF7408BE001ED39F401A7E017F089007E0
:10025E00D2E0FCA3E0FD1DBDFF011C1200038E5871
:10026E008F59801F9007D2E0FEA3E0FF7408126939
:10027E00BE8F048E057E017F08CDCCCD1200038E7D
:10028E00588F59AE5AAF5B7411D39F74019E5003B1
:10029E0002036EA2F9B3500302036BE55B455A707D
:1002AE000375A3D2AE5AAF5B74016F4E700375A384
:1002BE0000AE5AAF5B74026F4E700D9007D3E075AF
:1002CE00F002A4FDACF08DA3AE5AAF5B74036F4E7B
:1002DE00700375A300AE5AAF5B74046F4E70037556
:1002EE00A300AE5AAF5B74056F4E700375A300AEDC
:1002FE005AAF5B74066F4E700375A300AE5AAF5BB8
:10030E0074076F4E700375A300AE5AAF5B74086F1F
:10031E004E700375A300AE5AAF5B7408BE00039F08
:10032E005016AC58AD59ED2FFFEC3EFE90008912E1
:10033E0069A1E5A3F075A300AE5AAF5BEFB4100947
:10034E00EEB40105741412695AAE5AAF5BEFB410D5
:10035E0007EEB4010375F80D785A1269CE020291B8
:10036E0022755B00755A0075F809AE5AAF5B7417AB
:10037E00BE0004D39F5003020447A2F9B3500302F8
:10038E000444E55B455A700375A3D2AE5AAF5B7455
:10039E00016F4E700375A300AE5AAF5B74026F4EC1
:1003AE00700D9007D3E075F002A4FDACF08DA3AEF6
:1003BE005AAF5B74036F4E700375A300AE5AAF5BFA
:1003CE0074046F4E700375A300AE5AAF5B74056F65
:1003DE004E700375A300AE5AAF5B74066F4E70037A
:1003EE0075A300AE5AAF5B74076F4E700375A30012
:1003FE00AE5AAF5B74086F4E700375A300AE5AAF62
:10040E005B7408BE00039F500C90006B1269A1E54F
:10041E00A3F075A300AE5AAF5B74166F4E700574E1
:10042E001412695AAE5AAF5B74166F4E700375F89C
:10043E000D785A1269CE0203782290005DE0B4ABBB
:10044E000280030204E2755B00755A0075F809AE6E
:10045E005AAF5B7412BE007CD39F4078A2F9B340B2
:10046E0070E55B455A700375A382AE5AAF5B74019B
:10047E006F4E700375A300AE5AAF5B74026F4E7071
:10048E000D9007D3E075F002A4FDACF08DA3AE5A2B
:10049E00AF5B74036F4E700375A300AE5AAF5B74FF
:1004AE0003BE00039F50099000701269A1E0F5A3EE
:1004BE00AE5AAF5B74116F4E7005741412695AAE5A
:1004CE005AAF5B74116F4E700375F80D785A12693E
:1004DE00CE02045D229007DDE4F074649007D2F83A
:1004EE00E4F0E8A3F012036F74C89007D2F8E4F0BA
:1004FE00E8A3F0900077E0B4371A900074E0900013
:10050E006BF0900075E090006CF0900076E090003B
:10051E006DF080469007DD7401F074659007D2F897
:10052E00E4F0E8A3F012036F74C89007D2F8E4F079
:10053E00E8A3F0900077E0B4371A900074E09000D2
:10054E006BF0900075E090006CF0900076E09000FB
:10055E006DF0800674029007DDF09007DEE4F07413
:10056E00669007D2F8E4F0E8A3F012036F74C89017
:10057E0007D2F8E4F0E8A3F0900076E0B4371290DA
:10058E000074E0900065F0900075E090006EF080D1
:10059E00769007DE7401F074679007D2F8E4F0E805
:1005AE00A3F012036F74C89007D2F8E4F0E8A3F03A
:1005BE00900076E0B43712900074E0900065F090F1
:1005CE000075E090006EF0803E74029007DEF074CD
:1005DE00689007D2F8E4F0E8A3F012036F74C890A5
:1005EE0007D2F8E4F0E8A3F0900076E0B43712906A
:1005FE000074E0900065F0900075E090006EF08061
:10060E000674039007DEF022E54D64046006E5995A
:10061E0064FF6002802AA2324004D2328020E54D6F
:10062E00600874E6254D900061F0754D00E54C6054
:10063E000874F0254C900061F0754C00C2328002B7
:10064E00C232E54D9033F8F8282873754D00E599C0
:10065E00B4FF03754C01E599B4FE03754C02E599A0
:10066E00B4FD03754C03E599B4FC03754C04E59990
:10067E00B4FA03754C05E599B4FB06754D01123DB0
:10068E00C9E599B4F906754D04123DC9E599D3949F
:10069E00E54007E599C394F04002801685994E75A2
:1006AE004D027E017F00E54EC394E612697A8E31CB
:1006BE008F329007D6E4F0A3F0E599D394C44007A7
:1006CE00E599C394E64002802885994E754D0374D2
:1006DE00E5C3954EF532753100AE31AF3290637091
:1006EE00126949E493F87401939007D6C8F0A3C831
:1006FE00F0D299020AB3900074E070429007D6E0EF
:10070E00FEA3E0FF74FFBE00039F5009EFC39446A3
:10071E00EE940640119007D6E0FEA3E0FFEFD394CF
:10072E006DEE940640139007D6E0FEA3E0FF900016
:10073E00921269A1E599F080038599728011900754
:10074E00D6E0FEA3E0FF9000921269A1E599F09029
:10075E0007D61269889007D6E0FEA3E0FFEFB4013A
:10076E0006EEB40702800302089B900792E0B43CA9
:10077E00028003020885C29C900074E0900130F064
:10078E00900075E090009FF0900076E09000BFF032
:10079E00900077E09000E8F0900078E0900094F000
:1007AE00900079E09000DAF090007AE09000F8F096
:1007BE0090007BE09000CCF090007CE09000EAF09E
:1007CE0090007DE090011AF012371E900086E090A6
:1007DE000101F0900087E09000B8F0900088E09062
:1007EE0000B9F074639007D2F8E4F0E8A3F074ABAC
:1007FE0090005DF012044890005DE4F07509647598
:10080E0008001200E3A21F4038757101E571D39400
:10081E0007502CE5719007D2F8E4F0E8A3F074AA23
:10082E0090005DF012010FE571C394075009750930
:10083E00647508001200E37871740126F650CD80BD
:10084E0036757108E571D3940E502CE5719007D270
:10085E00F8E4F0E8A3F074AA90005DF012010FE541
:10086E0071C3940E50097509647508001200E3787F
:10087E0071740126F650CD74C89007D2F8E4F0E8F2
:10088E00A3F0D29C754D00754C007599FB020AB30E
:10089E009007D6E0FEA3E0FFEF4E70068599307507
:1008AE002F009007D6E0FEA3E0FF74016F4E701B81
:1008BE00AC2FAD30AA31AB32ED2BFBEC3AFA8A06F7
:1008CE008B079000921269A1E599F09007D61269F4
:1008DE00889007D6E0FEA3E0FF74026F4E7021AC45
:1008EE002FAD3074566D4C7006E54E64E660028096
:1008FE0003123DC912371E854E99754D00754C0079
:10090E00020AB39007D6E0FEA3E0FF9000921269B0
:10091E00A1E599F09007D61269889007D6E0FEA35C
:10092E00E0FFAC31AD328F028E038C068D079063E3
:10093E00B2126949E493F9740193FEEAD39EEB99DE
:10094E004009854E99754D00754C00020AB390070B
:10095E00D6E0FEA3E0FF9000921269A1E599F09017
:10096E0007D61269889007D6E0FEA3E0FFEFB40029
:10097E0006EEB401028003020AB390006DE075F03A
:10098E0002A4FDACF08D71ED9000921269ACEDFAFF
:10099E00E0FBEA9000951269ACEBFAE0FBEA2BFA69
:1009AE0090006DE0B502028003020AA50DED9000E5
:1009BE00921269ACE571FDE0FAED9000961269AC09
:1009CE00EAFDE0FAEDC39AFD90006DE0B5050280F8
:1009DE0003020AA5E5719000941269ACE571FDE081
:1009EE00FAED9000971269ACEAFDE0FAED2AFD905F
:1009FE00006DE0B505028003020AA5E5719000982E
:100A0E001269ACFDE0FAED90006DE0F4042A90005E
:100A1E0074F0E5719000991269ACFDE0FAED90006A
:100A2E006DE0F4042A900075F0E57190009A126959
:100A3E00ACFDE0FAED90006DE0F4042A900076F043
:100A4E00E57190009B1269ACFDE0FAED90006DE04F
:100A5E00F4042A9007D2F8E4F0E8A3F074AB900007
:100A6E005DF01204487509647508001200E39007E2
:100A7E00D21269881204487509647508001200E3E1
:100A8E009007D21269881204487599F97509647530
:100A9E0008001200E380FE7599FF75096475080061
:050AAE001200E380FED0
:0F33F80002065902070402089E02091102095C2D
:100AB30022E54C903407F8282873020B989007D648
:100AC300E0FEA3E0FF9000631269A1E0F5999007AF
:100AD300D61269889007D6E0FEA3E0FF74116F4E2B
:100AE3007003754C00020B98856C99020B98900764
:100AF300D6E0FEA3E0FF9000921269A1E0F599EF22
:100B0300B40107EEB40703754C009007D612698849
:070B1300020B989007D7E0E8
:0F340700020ABD020AC0020AEB020AF1020B160A
:100B1A009035BAF82828738551998067855D998040
:100B2A0062855F99805D8563998058856599805350
:100B3A00856699804E856799804985689980449031
:100B4A000026E0F599803CA233B340077599FAC2B2
:100B5A00338017A224B3400575990F800B9000616A
:100B6A00E0F599900061E4F0C224801785699980C4
:100B7A0012856499800D856A9980087599FC8003AD
:030B8A00754C00A7
:1035BA00020B21020B26020B2B020B30020B3502E7
:1035CA000B3A020B3F020B44020B49020B51020B4E
:0D35DA0076020B7B020B80020B85020B8A30
:0B0B8D009007D612698880031235E73C
:03341600020B9511
:100B980022E5362559FFAE5850010E900092126991
:100BA800A1E0F537E5362559FFAE5850010E0FBFC5
:100BB80000010E9000921269A1E0F538853E3AE5F1
:100BC80037B538058537368041E538D39537401D28
:100BD800E538C395378539F0A4FFAEF0E53A8E04C1
:100BE8008F05FF12696AED2537F536801DE537C395
:100BF80095388539F0A4FFAEF0E53A8E048F05FFED
:100C080012696AEDF4042537F53622E538D39537AD
:100C1800401DE538C395378539F0A4FFAEF0E53AB5
:100C28008E048F05FF12696AED2537F536801DE5BC
:100C380037C395388539F0A4FFAEF0E53A8E048FB6
:100C480005FF12696AEDF4042537F53622900098FD
:100C5800E0B40170E56575F00A84FF7E008F36E523
:100C68006575F00A84ADF07C008D39753E0A7558BB
:100C780005755924E536C394115005120B99800661
:100C88009005C7E0F536E53690008BF0E56575F020
:100C98000A84FF7E008F36E56575F00A84ADF07C26
:100CA800008D39753E0A75580575595AE536C3944D
:100CB800115005120B9980069005FDE0F536E536D2
:100CC80090001EF022900098E0B4016AE56575F086
:100CD8000A84FF7E008F36E56575F00A84ADF07CE6
:100CE800008D39753E0A755805755936E536C39431
:100CF800115005120B9980069005D9E0F536853616
:100D08004AE56575F00A84FF7E008F36E56575F063
:100D18000A84ADF07C008D39753E0A755805755901
:100D280048E536C394115005120B9980069005EBDF
:100D3800E0F53685364B22E55D75F00484FF7E00CC
:100D48008F36E55D75F00484ADF07C008D39753E15
:100D580004755801755900E536C3943F5005120BC8
:100D68009980069001D1E0F53685362875270090E0
:100D78000060E075F020A4FFAEF09000E3E08E0480
:100D88008F05FF12696A8D369000CBE0D3955D50D0
:100D980003020E459000EFE0D3955D4010ED900101
:100DA800D21269ACE0F52A752900020E429000BA09
:100DB800E0D3955D4043E5369001D21269ACE0F589
:100DC80037E5369001F21269ACE0F5389000EFE0B3
:100DD800F404255DF5399000BAE0FE9000EFE0F4E8
:100DE800042EF53AE537B538058537368003120CF9
:100DF8001385362A7529008041E5369001F212697B
:100E0800ACE0F537E5369002121269ACE0F538909F
:100E180000BAE0F404255DF5399000CBE0FE9000BF
:100E2800BAE0F4042EF53AE537B53805853736804B
:100E380003120C1385362A752900020EEC9000F275
:100E4800E0D3955D5011E5369002521269ACE0F599
:100E58002A752900020EEC9000BBE0D3955D504343
:100E6800E5369002321269ACE0F537E53690025269
:100E78001269ACE0F5389000BBE0F404255DF53963
:100E88009000F2E0FE9000BBE0F4042EF53AE5375E
:100E9800B538058537368003120C1385362A75292F
:100EA800008041E5369002121269ACE0F537E5366C
:100EB8009002321269ACE0F5389000CBE0F40425DA
:100EC8005DF5399000BBE0FE9000CBE0F4042EF510
:100ED8003AE537B538058537368003120C13853661
:100EE8002A75290022900103E0F53B753E117558DB
:100EF80002755900AE50AF51E53B75F00FA4FDAC3B
:100F0800F0EDD39FEC9E4021E53B8E048F05FF1248
:100F1800696AED75F010A4FFAEF0E55D75F0118417
:100F2800FD7C00ED2FF53C800EE55D75F01184FF2A
:100F38007E00EF24F0F53C853C36E55D75F01184C4
:100F4800AFF07E008F39120B9985363DAE50AF5108
:100F5800900103E075F00FA4FDACF0EDD39FEC9E7B
:100F68004028755802755910853C36120B99853DF5
:100F780037853638AE50AF51E53B8E048F05FF12EA
:100F880069958D39853B3A120C13853628752700EB
:100F9800752A6475290022900103E0F53B753E111E
:100FA800755802755900AE50AF51E53B75F00FA466
:100FB800FDACF0EDD39FEC9E4021E53B8E048F0500
:100FC800FF12696AED75F010A4FFAEF0E55F75F0E9
:100FD8001184FD7C00ED2FF53C800EE55F75F01166
:100FE80084FF7E00EF24F0F53C853C36E55F75F024
:100FF8001184AFF07E008F39120B9985363DAE50C3
:10100800AF51900103E075F00FA4FDACF0EDD39F54
:10101800EC9E4028755802755910853C36120B997C
:10102800853D37853638AE50AF51E53B8E048F0588
:10103800FF1269958D39853B3A120C138536287550
:1010480027009000CDE0B40453E55D75F00484FFFB
:101058007E008F36E55D75F00484ADF07C008D3937
:10106800753E04755801755900E536C3943F50051F
:10107800120B9980069001D1E0F536AE27AF28E52E
:101088003612697A74648E048F05FF12696AAE2776
:10109800AF28EF2DFDEE3CFC8C278D28752A647552
:1010A800290022900098E0B40146E56575F00A84AD
:1010B800FF7E008F36E56575F00A84ADF07C008D03
:1010C80039753E0A755805755900E536C3941150AF
:1010D80005120B9980069005A3E0F536AE29AF2AD4
:1010E800E5362FFF50010E74641269BE8E298F2ACF
:1010F800900099E0B40146E56675F00A84FF7E0029
:101108008F36E56675F00A84ADF07C008D39753E42
:101118000A75580575596CE536C394115005120BBC
:1011280099800690060FE0F536AE29AF2AE5362FEE
:10113800FF50010E74641269BE8E298F2A9000A890
:10114800E0B40249E568C3944175F00584FF7E0068
:101158008F36E56875F00584ADF07C008D39753EF5
:1011680005755806755900E536C394135005120BDA
:101178009980069006A5E0F536AE29AF2AE5362F08
:10118800FF50010E74641269BE8E298F2A9000EAFE
:10119800E0B40202800302124AE55D75F01584FF8F
:1011A8007E008F36E55D75F01584ADF07C008D39D5
:1011B800753E157558037559F4E536C3940B5005FB
:1011C800120B998006900491E0F536E53675F0FF2C
:1011D800A4FFAEF09000EBE08E048F05FF12696A61
:1011E800ED900084F0E56475F078A4FFAEF074FF2C
:1011F8008E048F05FF12696A8C588D5974028C060B
:101208008D071200398F36AC58AD597404FF126936
:10121800958D39753E04755806755928E536C39479
:101228001D5005120B9980069006D7E0F536AE29B9
:10123800AF2AE5362FFF50010E74641269BE8E295D
:101248008F2A900097E0B4025DE55F75F064A4FF13
:10125800AEF074081200398E5A8F5B74058E048FB5
:1012680005FF12696A8D36AE5AAF5B74058E048F1E
:1012780005FF1269958D39753E057558057559DE56
:10128800E536C394135005120B998006900683E047
:10129800F536AE29AF2AE5362FFF50010E746412D9
:1012A80069BE8E298F2A9000D9E0703C900060E0DA
:1012B80075F00584FF7E008F36900060E075F005BC
:1012C80084ADF07C008D39753E057558057559C09B
:1012D800E536C3941D5005120B99800690066FE001
:1012E800F536E53690008CF0229000A0E0B40117A6
:1012F8009007D9E0252AFFAE2950010E9000F4E0AE
:101308001269BE8E298F2A900118E0B40114900149
:1013180019E0A850B8000495515007E55DC3955EE3
:10132800400280129000C2E0252AFFAE2950010E2B
:101338008E298F2A802F9000A0E0B40316A226B32E
:10134800B350109007DCE0C39405A850B800069588
:1013580051400280109000C2E0252AFFAE295001BA
:101368000E8E298F2A90009AE0B40202800302159B
:101378004D90009DE0602FE565D39446402890008D
:101388001FE0FEA3E0FF9000D8E075F003A4FDACD9
:10139800F0EFD39DEE9C400E9000FCE0A850B80002
:1013A80005D39551500302154D9000E5E0855DF099
:1013B800A4FFAEF0740512697A74071200398E58CA
:1013C8008F599000A4E0A850B8000495515012908D
:1013D80000A5E075F002A4FDACF0EFC39DEE9C40C3
:1013E8000302154DE55D75F00B84FF7E0090062223
:1013F8001269A1FEE0FFEE90009CE0FEEF8E0088EF
:10140800F0A4FFAEF074648E048F05FF12696A8C35
:10141800588D59900060E075F018A4FFAEF0900068
:10142800E3E08E048F05FF12696A8C068D0790062B
:101438003A1269A1AE58AF59E012697A74648E0401
:101448008F05FF12696A8C588D59E563A858B80052
:1014580077D395594072E563C39559FFE49558FED3
:101468008E588F597428BE00039F500C75592875E3
:101478005800740D900061F0AE58AF5990009DE08F
:1014880012697A74288E048F05FF12696A8C588D48
:1014980059AE27AF28740A8E048F05FF12696A8D2A
:1014A800068C07AC58AD59CFCECF120003740A8E04
:1014B800048F05FF12696A8C588D59AE27AF281220
:1014C80069C68E278F28807DE563A858B8000495E3
:1014D800595072AE58AF59E5631269BE8E588F598C
:1014E8007428BE00039F500C755928755800740D58
:1014F800900061F0AE58AF5990009DE012697A747F
:10150800288E048F05FF12696A8C588D59AE27AF53
:1015180028740A8E048F05FF12696A8D068C07AC41
:1015280058AD59CFCECF120003740A8E048F05FF31
:1015380012696A8C588D59AE27AF28EF2DFDEE3C05
:10154800FC8C278D28229000F8E0B4026AE55D75CE
:10155800F00884FF7E008F36E55D75F00884ADF0F5
:101568007C008D39753E087558017559E0E536C31C
:10157800943F5005120B998006900291E0F536854C
:10158800362C752B00AE2BAF2CAC29AD2A120003DC
:1015980074648E048F05FF12696A8C2B8D2C900061
:1015A80095E08C068D0712697A74648E048F05FFA6
:1015B80012696A8C2B8D2CAE27AF28AC29AD2A1264
:1015C800000374648E048F05FF12696A8C278D28C6
:1015D800900095E08C068D0712697A74648E048FEA
:1015E80005FF12696A8C278D28A207401DAE50AFEF
:1015F800517405BE00039F5002D207E55FD394CC17
:101608004008D2017411900061F09000F7E0B40234
:10161800089000F9E0640160028035AE27AF28E544
:101628006912697A74E78E048F05FF12696A8C273C
:101638008D289000F8E0B40217AE2BAF2CE56912A4
:10164800697A74E78E048F05FF12696A8C2B8D2CDA
:101658009000B7E05402601B9000AEE0A850B800BC
:1016680012D39551400DA207B3B35007E55FC39459
:101678009A40028028AE34AF359000ACE075F00295
:10168800A4FDACF0EF2DFDEE3CFC74022DFD5001E5
:101698000CE55FBC0007D39D4003754201855F35AB
:1016A800753400E542700302179190010AE0C39572
:1016B80042500302178390011AE0C394025076E562
:1016C8006575F00A84FF7E009005921269A1E0F525
:1016D80059755800AE58AF599000ADE012697A7448
:1016E800648E048F05FF12696A8C5A8D5B90010A1B
:1016F800E004C395428C068D0712697A90010AE0CE
:101708008E048F05FF12696A8C5A8D5BAE27AF284D
:10171800EF2DFDEE3CFC8C278D289000F8E0B402FC
:1017280012AE2BAF2CAA5AAB5BEF2BFBEE3AFA8A20
:101738002B8B2C804690010AE004C39542854AF021
:10174800A4FFAEF090010AE08E048F05FF12696ACB
:101758008C5A8D5BAE27AF28EF2DFDEE3CFC8C2715
:101768008D289000F8E0B40212AE2BAF2CAA5AAB29
:101778005BEF2BFBEE3AFA8A2B8B2C054290010A81
:10178800E0C3954250037542009000B7E0540160F1
:101798001B9000ABE0A850B80012D39551400DA2A1
:1017A80007B3B35007E55DC394CC40028025900091
:1017B800A9E075F003A4FFAEF0E53F2FFF50010E3E
:1017C80074032FFF50010EE55DBE0007D39F400351
:1017D800754301855D3FE54370030218C490010B12
:1017E800E0C3954350030218B690011AE0C394026F
:1017F8005076E56575F00A84FF7E009005921269BF
:10180800A1E0F559755800AE58AF599000AAE012FA
:10181800697A74648E048F05FF12696A8C5A8D5B2D
:1018280090010BE004C395438C068D0712697A90EA
:10183800010BE08E048F05FF12696A8C5A8D5BAE2E
:1018480027AF28EF2DFDEE3CFC8C278D289000F863
:10185800E0B40212AE2BAF2CAA5AAB5BEF2BFBEE17
:101868003AFA8A2B8B2C804690010BE004C39543EF
:10187800854BF0A4FFAEF090010BE08E048F05FFBE
:1018880012696A8C5A8D5BAE27AF28EF2DFDEE3CAE
:10189800FC8C278D289000F8E0B40212AE2BAF2CF8
:1018A800AA5AAB5BEF2BFBEE3AFA8A2B8B2C05433B
:1018B80090010BE0C39543500375430090010DE080
:1018C8002528FFAE2750010E8E278F289000BCE0F8
:1018D800A827B80004952850099000BCE0F52875A1
:1018E80027009000F8E0B4020D9000BCE0A82BB8E7
:1018F8000006952C400280099000BCE0F52C752B61
:1019080000229000F8E0B401028003021A15A20731
:10191800B35003021A139000C3E0B40168AE27AFB6
:1019280028AC50AD51120003743C8E048F05FF1291
:10193800696A9000D3E0BC00109D400D9000D5E08E
:10194800A827B8000495285002D202AE27AF28ACC9
:1019580050AD51120003743C8E048F05FF12696A62
:101968009000D3E0C3940ABC0015D39D40119000A9
:10197800D5E0C39405A827B80005D3952850028060
:1019880002C2028068AE27AF28AC50AD51120003E6
:1019980074788E048F05FF12696A9000D3E0BC004A
:1019A800109D400D9000D5E0A827B8000495285058
:1019B80004D2028038AE27AF28AC50AD51120003D4
:1019C80074788E048F05FF12696A9000D3E0C3947F
:1019D8000ABC0015D39D40119000D5E0C39405A81A
:1019E80027B80005D3952850028002C202A202B38C
:1019F8004019AE27AF289000D4E012697A74648E3B
:101A0800048F05FF12696A8C278D288002C202A202
:101A180000B34006A201B3B35009900025E4F0A337
:101A2800F08024AE27AF287400D39F74019E400C29
:101A3800900025E527F0A3E528F0800B74FF9000BF
:101A480025F8E4F0E8A3F09000DAE0D39402400C23
:101A58009000C5E07006A207B3B34002801AAE2713
:101A6800AF28740212697A8E278F28AE2BAF2C7498
:101A78000212697A8E2B8F2C9000C3E0B4011AAE43
:101A880027AF28740212697A8E278F28AE2BAF2CC5
:101A9800740212697A8E2B8F2CAE27AF28745E12CF
:101AA800697A740A8E048F05FF12696A8C278D285B
:101AB8009000F8E0B40217AE2BAF2C745E12697A6E
:101AC800740A8E048F05FF12696A8C2B8D2CAE2741
:101AD800AF287402BE000AD39F40067528027527F6
:101AE80000AE2BAF2C7402BE000AD39F4006752CA3
:101AF80002752B00900023E527F0A3E528F022903B
:101B08000060E09003921269ACE0F5407541649082
:101B18000060E0FE9000CEE0D39E4037E55D75F0B2
:101B28000884FF7E008F36E55D75F00884ADF07C93
:101B3800008D39753E08755803755996E536C39476
:101B48001F5005120B998006900447E0F53685363C
:101B5800418035E55D75F00884FF7E008F36E55DD0
:101B680075F00884ADF07C008D39753E0875580312
:101B78007559B6E536C3941F5005120B9980069027
:101B88000467E0F53685364122900104E0F53B759F
:101B98003E11755804755900AE50AF51E53B75F0CC
:101BA8000FA4FDACF0EDD39FEC9E4021E53B8E04E5
:101BB8008F05FF12696AED75F010A4FFAEF0E55DC0
:101BC80075F01184FD7C00ED2FF53C800EE55D7508
:101BD800F01184FF7E00EF24F0F53C853C36E55D8E
:101BE80075F01184AFF07E008F39120B9985363D60
:101BF800AE50AF51900104E075F00FA4FDACF0EDCC
:101C0800D39FEC9E4028755804755910853C3612B0
:101C18000B99853D37853638AE50AF51E53B8E047C
:101C28008F05FF1269958D39853B3A120C1385365D
:101C38004075416422900104E0F53B753E117558EA
:101C480004755900AE50AF51E53B75F00FA4FDACDB
:101C5800F0EDD39FEC9E4021E53B8E048F05FF12EB
:101C6800696AED75F010A4FFAEF0E55F75F01184B8
:101C7800FD7C00ED2FF53C800EE55F75F01184FFCB
:101C88007E00EF24F0F53C853C36E55F75F0118465
:101C9800AFF07E008F39120B9985363DAE50AF51AB
:101CA800900104E075F00FA4FDACF0EDD39FEC9E1D
:101CB8004028755804755910853C36120B99853D96
:101CC80037853638AE50AF51E53B8E048F05FF128D
:101CD80069958D39853B3A120C13853640754164F8
:101CE8009000FFE0B40479900060E0FE9000CEE040
:101CF800D39E4037E55D75F00884FF7E008F36E59A
:101D08005D75F00884ADF07C008D39753E08755816
:101D180003755996E536C3941F5005120B99800632
:101D2800900447E0F5368536418035E55D75F00865
:101D380084FF7E008F36E55D75F00884ADF07C0089
:101D48008D39753E087558037559B6E536C3941F25
:101D58005005120B998006900467E0F536853641E8
:101D680022900098E0B4013BE56575F00A84FF7E97
:101D7800008F36E56575F00A84ADF07C008D397505
:101D88003E0A755805755912E536C3941150051267
:101D98000B9980069005B5E0F536E5412536C394E4
:101DA80064F541900099E0B4013BE56675F00A845A
:101DB800FF7E008F36E56675F00A84ADF07C008DF5
:101DC80039753E0A75580575597EE536C394115024
:101DD80005120B998006900621E0F536E541253677
:101DE800C39464F541E5402541F5339000A0E0B483
:101DF80002109007D8E02533FE9000F4E0F4042E9A
:101E0800F5339000F7E0D394014040E569C394E7C7
:101E1800501D74E7C39569FE9007DAE08E00F5F06F
:101E2800E884FF7E008F36E5332536F533801CE5E0
:101E380069C394E7FE9007DAE08E00F5F0E884FFC6
:101E48007E008F36E533C39536F533A2074006E5A5
:101E5800402464F533E533D394644009E533C394EF
:101E680064F53380037533009000D0E0C395335098
:101E7800069000D0E0F53322D20090008AE0A85006
:101E8800B800049551504190008AE0A850B8000469
:101E98009551500375330F90008AE004A850B8009C
:101EA800049551500375330A90008AE02402A85023
:101EB800B8000495515005753305C20090008AE0BA
:101EC80060067409900061F0C2367E017F009000C0
:101ED800D6E012697A9000E5E08E048F05FF12695A
:101EE8006AE55DBC0017D39D40139000DFE0B402A3
:101EF80004D2368002C200740A900061F09000D7C4
:101F0800E0C3956550159000E9E0A850B800049525
:101F1800515002C200740B900061F0E565C39464EF
:101F2800501D90012FE0600D90012FE0A850B800DF
:101F380006955140028008C200740B900061F0A21F
:101F4800004003753305900118E0B401149001199D
:101F5800E0A850B8000495515007E55DC3955E4070
:101F68000280089000C1E0F533803A9000A0E0B408
:101F78000306A226B3B34002802B9007DCE0C3948B
:101F880005A850B800049551500C9000C1E0F533F5
:101F9800740C900061F09007DCE0A850B80004953C
:101FA800515002C20085336A900092E02533FE90BA
:101FB8000060E075F01E84FC7F00EE2CF533229063
:101FC8000060E075F00584FF7E008F36900060E0C9
:101FD80075F00584ADF07C008D39753E05755803A4
:101FE8007559D69000E3E01475F00584FF7E00E58E
:101FF80036BE00039F5005120B99800BE5369004FE
:10200800681269ACE0F536E5369007DBF09007DB3F
:10201800E0FE9000D2E0C39E50089000D2E0900706
:10202800DBF022E56575F00A84FF7E0090059212C8
:1020380069A1E0F545E545D394644010E545C394AE
:102048006475F00F84FF7E008F458003754500900E
:1020580000B5E02545F545229007CCE0FEA3E0FF5A
:102068007404120039E55D12697A740F8E048F05C5
:10207800FF12696A9007CAECF0A3EDF09000A8E09F
:10208800B40262E568C3944175F00584FF7E008F51
:1020980036E56875F00584ADF07C008D39753E0530
:1020A800755806755914E536C394175005120B99DF
:1020B80080069006B9E0F5369007CAE0FEA3E0FF77
:1020C800740A8E048F05FF12696AE5368C068D073F
:1020D80012697A740A8E048F05FF12696A9007CA1A
:1020E800ECF0A3EDF09007CAE0FEA3E0FF9007D064
:1020F800E0FCA3E0FDEDD39FEC9E400F9007D0E0FD
:10210800F8A3E09007CAC8F0A3C8F0229006D9E067
:10211800903419F8282873804C85517180479000B5
:10212800E5E0855DF0A4FFAEF074081200398F7108
:102138008033855F71802E85657180298566718001
:1021480024856771801F856871801A85697180157B
:102158008564718010856371800B856A7180069033
:052168000026E0F57106
:1034190002211F02212102212602213A02213F0213
:10342900214402214902214E02215302215802213D
:073439005D02216202216720
:10216D009006DAE0FE9006DBE0D39E404B9006D958
:10217D00E0B404189006DBE0C395715002D22790AD
:10218D0006DAE0D395714002C227802A9006DAE084
:10219D00C3957150099006DBE0D395715002800212
:1021AD00D2279006DAE0D3957150099006DBE0C393
:1021BD0095715002C227802A9006DAE0D3957140BE
:1021CD00099006DBE0C3957140028002C22790069C
:1021DD00DAE0C3957140099006DBE0D395714002BA
:1021ED00D227229006DDE0903440F8282873804CE9
:1021FD0085517180479000E5E0855DF0A4FFAEF05C
:10220D0074081200398F718033855F71802E85655A
:10221D007180298566718024856771801F8568713D
:10222D00801A856971801585647180108563718050
:0C223D000B856A718006900026E0F571A8
:103440000221FB0221FD02220202221602221B029D
:10345000222002222502222A02222F0222340222C4
:073460003902223E02224363
:102249009006DEE0FE9006DFE0D39E405F9006DD5B
:10225900E0B404189006DFE0C395715002D22890CB
:1022690006DEE0D395714002C228803E9006DEE08A
:10227900C3957150099006DFE0D395715002800231
:10228900D2289006DEE0D3957150099006DFE0C3AD
:1022990095715002C2289006DDE0B401099000F161
:1022A900E0D3955F50028002C228802A9006DEE0C2
:1022B900D3957140099006DFE0C395714002800211
:1022C900C2289006DEE0C3957140099006DFE0D38D
:1022D90095714002D228229006E1E0903467F828EF
:1022E9002873804C85517180479000E5E0855DF049
:1022F900A4FFAEF074081200398F718033855F71C5
:10230900802E856571802985667180248567718035
:102319001F856871801A85697180158564718010BF
:10232900856371800B856A718006900026E0F571DE
:103467000222EB0222ED0222F202230602230B02C2
:10347700231002231502231A02231F0223240223E7
:073487002902232E0223336A
:102339009006E2E0FE9006E3E0D39E404B9006E172
:10234900E0B404189006E3E0C395715002D22990D5
:1023590006E2E0D395714002C229802A9006E2E0A4
:10236900C3957150099006E3E0D39571500280023C
:10237900D2299006E2E0D3957150099006E3E0C3B3
:1023890095715002C229802A9006E2E0D3957140E6
:10239900099006E3E0C3957140028002C2299006C4
:1023A900E2E0C3957140099006E3E0D395714002DC
:1023B900D229229006E5E090348EF8282873804CC3
:1023C90085517180479000E5E0855DF0A4FFAEF08E
:1023D90074081200398F718033855F71802E85658D
:1023E9007180298566718024856771801F85687170
:1023F900801A856971801585647180108563718083
:0C2409000B856A718006900026E0F571DA
:10348E000223C70223C90223CE0223E20223E7024C
:10349E0023EC0223F10223F60223FB022400022472
:0734AE000502240A02240FAD
:102415009006E6E0FE9006E7E0D39E404B9006E589
:10242500E0B404189006E7E0C395715002D22A90F3
:1024350006E6E0D395714002C22A802A9006E6E0BE
:10244500C3957150099006E7E0D39571500280025B
:10245500D22A9006E6E0D3957150099006E7E0C3CD
:1024650095715002C22A802A9006E6E0D395714004
:10247500099006E7E0C3957140028002C22A9006E2
:10248500E6E0C3957140099006E7E0D395714002F7
:10249500D22A229006E9E09034B5F8282873804CBA
:1024A50085517180479000E5E0855DF0A4FFAEF0B1
:1024B50074081200398F718033855F71802E8565B0
:1024C5007180298566718024856771801F85687193
:1024D500801A8569718015856471801085637180A6
:0C24E5000B856A718006900026E0F571FE
:1034B5000224A30224A50224AA0224BE0224C302D4
:1034C50024C80224CD0224D20224D70224DC0224FB
:0734D500E10224E60224EBF2
:1024F1009006EAE0FE9006EBE0D39E404B9006E9A1
:10250100E0B404189006EBE0C395715002D22B9011
:1025110006EAE0D395714002C22B802A9006EAE0D8
:10252100C3957150099006EBE0D39571500280027A
:10253100D22B9006EAE0D3957150099006EBE0C3E7
:1025410095715002C22B802A9006EAE0D395714022
:10255100099006EBE0C3957140028002C22B900600
:10256100EAE0C3957140099006EBE0D39571400212
:10257100D22B229006EDE09034DCF8282873804CB1
:1025810085517180479000E5E0855DF0A4FFAEF0D4
:1025910074081200398F718033855F71802E8565D3
:1025A1007180298566718024856771801F856871B6
:1025B100801A8569718015856471801085637180C9
:0C25C1000B856A718006900026E0F57121
:1034DC0002257F02258102258602259A02259F025C
:1034EC0025A40225A90225AE0225B30225B8022582
:0734FC00BD0225C20225C735
:1025CD009006EEE0FE9006EFE0D39E404B9006EDB8
:1025DD00E0B404189006EFE0C395715002D22C9030
:1025ED0006EEE0D395714002C22C802A9006EEE0F3
:1025FD00C3957150099006EFE0D39571500280029A
:10260D00D22C9006EEE0D3957150099006EFE0C301
:10261D0095715002C22C802A9006EEE0D395714040
:10262D00099006EFE0C3957140028002C22C90061E
:10263D00EEE0C3957140099006EFE0D3957140022D
:10264D00D22C229006F1E0903503F8282873804CA7
:10265D0085517180479000E5E0855DF0A4FFAEF0F7
:10266D0074081200398F718033855F71802E8565F6
:10267D007180298566718024856771801F856871D9
:10268D00801A8569718015856471801085637180EC
:0C269D000B856A718006900026E0F57144
:1035030002265B02265D02266202267602267B02E3
:10351300268002268502268A02268F022694022608
:073523009902269E0226A377
:1026A9009006F2E0FE9006F3E0D39E404B9006F1CF
:1026B900E0B404189006F3E0C395715002D22D904E
:1026C90006F2E0D395714002C22D802A9006F2E00D
:1026D900C3957150099006F3E0D3957150028002B9
:1026E900D22D9006F2E0D3957150099006F3E0C31C
:1026F90095715002C22D802A9006F2E0D39571405F
:10270900099006F3E0C3957140028002C22D90063C
:10271900F2E0C3957140099006F3E0D39571400248
:10272900D22D229006F5E090352AF8282873804C9E
:1027390085517180479000E5E0855DF0A4FFAEF01A
:1027490074081200398F718033855F71802E856519
:102759007180298566718024856771801F856871FC
:10276900801A85697180158564718010856371800F
:0C2779000B856A718006900026E0F57167
:10352A0002273702273902273E022752022757026B
:10353A00275C02276102276602276B02277002278F
:07354A007502277A02277FBA
:102785009006F6E0FE9006F7E0D39E404B9006F5E6
:10279500E0B404189006F7E0C395715002D22E906C
:1027A50006F6E0D395714002C22E802A9006F6E027
:1027B500C3957150099006F7E0D3957150028002D8
:1027C500D22E9006F6E0D3957150099006F7E0C336
:1027D50095715002C22E802A9006F6E0D39571407D
:1027E500099006F7E0C3957140028002C22E90065B
:1027F500F6E0C3957140099006F7E0D39571400264
:10280500D22E229006F9E0903551F8282873804C95
:1028150085517180479000E5E0855DF0A4FFAEF03D
:1028250074081200398F718033855F71802E85653C
:102835007180298566718024856771801F8568711F
:10284500801A856971801585647180108563718032
:0C2855000B856A718006900026E0F5718A
:1035510002281302281502281A02282E02283302F3
:10356100283802283D02284202284702284C022816
:073571005102285602285BFD
:102861009006FAE0FE9006FBE0D39E404B9006F9FD
:10287100E0B404189006FBE0C395715002D22F908A
:1028810006FAE0D395714002C22F802A9006FAE041
:10289100C3957150099006FBE0D3957150028002F7
:1028A100D22F9006FAE0D3957150099006FBE0C350
:1028B10095715002C22F802A9006FAE0D39571409B
:1028C100099006FBE0C3957140028002C22F900679
:1028D100FAE0C3957140099006FBE0D3957140027F
:1028E100D22F229006FDE0903578F8282873804C8D
:1028F10085517180479000E5E0855DF0A4FFAEF061
:1029010074081200398F718033855F71802E85655F
:102911007180298566718024856771801F85687142
:10292100801A856971801585647180108563718055
:0C2931000B856A718006900026E0F571AD
:103578000228EF0228F10228F602290A02290F027E
:10358800291402291902291E02292302292802299D
:073598002D02293202293740
:10293D009006FEE0FE9006FFE0D39E404B9006FD14
:10294D00E0B404189006FFE0C395715002D23090A8
:10295D0006FEE0D395714002C230802A9006FEE05B
:10296D00C3957150099006FFE0D395715002800216
:10297D00D2309006FEE0D3957150099006FFE0C36A
:10298D0095715002C230802A9006FEE0D3957140B9
:10299D00099006FFE0C3957140028002C230900697
:1029AD00FEE0C3957140099006FFE0D3957140029A
:1029BD00D23022AE2DAF2E74F5D39F74019E4008F8
:1029CD00782D1269CE022ADA752E01752D00AE50C2
:1029DD00AF51E545BE000DD39F40099000C7E0D330
:1029ED00954640028023754600E545C39551F57126
:1029FD009000CAE0D395444008E5442571F5448024
:102A0D00069000CAE0F544800205469000A3E0D38D
:102A1D00955F401CE55DC3955E4015AE50AF51E529
:102A2D0045BE00039F50099000C8E0D39547400272
:102A3D00806E9007DFE0A850B800049551500375E3
:102A4D0049009007DFE0A850B8000BD39551400620
:102A5D00E5519007DFF0E5497041E551C39545F526
:102A6D0071E571D3940540037571059000C9E0C3FC
:102A7D0095445007E571C3954440028009E544C370
:102A8D009571F54480069000C9E0F5449000C9E0C9
:102A9D00D3954440069000C9E0F544754700800287
:102AAD000547E54970169000A3E0C3955F500DE50D
:102ABD00452405A850B8000695514002800F90009E
:102ACD00B6E0F54475490174789007DFF022AE2D1C
:102ADD00AF2E74E9D39F74039E4008782D1269CEF2
:102AED00022C79752E01752D00754432A231402AC4
:102AFD007544199000B6E075F002A4FFAEF0E546FE
:102B0D00BE0006D39F4002D2310546754903747845
:102B1D009007DFF0754800022C68AE50AF51E545C7
:102B2D006F4E7003022C68E545BE000DD39F400922
:102B3D009000C7E0D395464002800F754600E549E9
:102B4D00C394035003754419800DE545C39551F5A4
:102B5D0071E5462571F5469000A3E0D3955F400ED3
:102B6D009007DFE0A850B80007D395514002800CC4
:102B7D0005489000B6E0B54803754900E549B40332
:102B8D0006A207B3B34002800A0548E548B43C03EA
:102B9D00754902E549B402299007DFE0A850B80055
:102BAD000ED395514009E5519007DFF0754800901F
:102BBD0000A3E0C3955F500975480074789007DF56
:102BCD00F0E549705A9000A3E0D3955F401CE55D98
:102BDD00C3955E4015AE50AF51E545BE00039F5005
:102BED00099000C8E0D395474002800875470075ED
:102BFD00444B8028E551C39545F571E571D3940596
:102C0D0040037571059000A3E0D3955F4008E5473B
:102C1D002571F5478006E5472406F547754800E51B
:102C2D004970169000A3E0C3955F500DE54524054E
:102C3D00A850B80006955140028003754901E54939
:102C4D00B4011875441905489000B6E0B5480675ED
:102C5D00490275480074789007DFF0E54475F00A75
:102C6D00A4FFAEF09007D4EEF0A3EFF022E56D9047
:102C7D00359FF828287390009BE07003022E289052
:102C8D0000D1E0B401028003022D7890005EE0B522
:102C9D005C028003022D757E017F00E5BE12697A0C
:102CAD00E5BD2FFF50010E8E588F59741012697AA1
:102CBD00900089E08E048F05FF12696A9007E0ECA1
:102CCD00F0A3EDF0E56960089000F7E064026002A2
:102CDD0080269000F9E0B4011F9007E0E0FEA3E02C
:102CED00FF74E712697AE5698E048F05FF12696A30
:102CFD009007E0ECF0A3EDF090009BE0B40227907C
:102D0D0007E2E0FEA3E0FF9007E0E0FCA3E0FDEFAB
:102D1D002DFDEE3CFC74018C068D071200399007D9
:102D2D00E0EEF0A3EFF09007E0E0FEA3E0FF9007E8
:102D3D00E2E0FCA3E0FDEDD39FEC9E4004D2348095
:102D4D0002B2349007E0E0F8A3E09007E2C8F0A3E8
:102D5D00C8F09000CDE064016006A234B3B3400228
:102D6D0080069007E1E0F55D022E26D2347E017FCC
:102D7D0000E5BE12697AE5BD2FFF50010E8E588F0A
:102D8D0059741012697A900089E08E048F05FF1234
:102D9D00696A9007E0ECF0A3EDF0E569600890003A
:102DAD00F7E06402600280269000F9E0B4011F9004
:102DBD0007E0E0FEA3E0FF74E712697AE5698E048F
:102DCD008F05FF12696A9007E0ECF0A3EDF090001B
:102DDD009BE0B402279007E2E0FEA3E0FF9007E03E
:102DED00E0FCA3E0FDEF2DFDEE3CFC74018C068DA7
:102DFD00071200399007E0EEF0A3EFF09007E0E046
:102E0D00F8A3E09007E2C8F0A3C8F09000CDE0640D
:102E1D000160069007E1E0F55D8003755D009000AF
:102E2D0097E07006756D01022C7A75BB180233F3AD
:102E3D00900097E07003022FC97E017F00E5BE125E
:102E4D00697AE5BD2FFF50010E8E588F599000DD28
:102E5D00E0B4010F7E0F7FFFAC58AD591269C68EDD
:102E6D00588F59900102E0B40245AE58AF59900009
:102E7D002FE0FCA3E0FDEDD39FEC9E400A90002FC8
:102E8D00E558F0A3E559F0AE58AF59900031E0FC8C
:102E9D00A3E0FDEFD39DEE9C400A900031E558F084
:102EAD00A3E559F0AE58AF5974041200398F5F90F5
:102EBD000102E0704CAE58AF5990002FE0FCA3E03A
:102ECD00FDEFD39DEE9C40091269C68E588F598037
:102EDD0006755900755800AE58AF59741012697ABD
:102EED00900086E08E048F05FF12696A8C588D590B
:102EFD0074FFBC0009D39D400585595F8003755F44
:102F0D00FE9000CDE0B401028003022FC7A207B3EB
:102F1D00B3500E9000A1E0A850B80005D3955150C4
:102F2D0003022FBC9000A2E075F019A4FFAEF09043
:102F3D0000E5E08E048F05FF12696A9000DEE085E2
:102F4D005FF0A4FFAEF074648D028C038E048F05C8
:102F5D00FF12696AEA2DFDEB3CFC8C588D59E56931
:102F6D00600F9000F7E0B402089000F9E064016092
:102F7D00028017AE58AF5974E712697AE5698E046D
:102F8D008F05FF12696A8C588D59AE58AF5990074D
:102F9D00E0E0FCA3E0FDEDD39FEC9E400585595D7F
:102FAD00800BA234B340069007E1E0F55D800BA2E3
:102FBD0034B340069007E1E0F55D8003755F009046
:102FCD00009AE07006756D02022C7A75BB190233FA
:102FDD00F390009AE0700302307EE55CD3954F408C
:102FED000302307C90002DE0FEA3E0FFE563126943
:102FFD00BE90002DEEF0A3EFF07E017F00E5BE1236
:10300D00697AE5BD2FFF50010E8E588F599001073B
:10301D00E07013740A12697A74518E048F05FF12D1
:10302D00696A8D638019AE58AF59740A12697A8F27
:10303D00048E057E017F95CDCCCD1268688F63E53A
:10304D0063D39464400375636490002DE0FEA3E0A8
:10305D00FFE5632FFF50010E90002DEEF0A3EFF072
:10306D0090009EE0048E048F05FF12696A8D6380C7
:10307D00037563329000EAE07006756D03022C7AD9
:10308D0075BB130233F39000EAE0604A7E017F00C6
:10309D00E5BE12697AE5BD2FFF50010E8E588F598E
:1030AD0074041200398F649000ECE08564F0A4FD87
:1030BD00ACF07464FF12696A8D649000EBE0856476
:1030CD00F0A4FFAEF074FF8E048F05FF12696AED58
:1030DD00900085F08003756400900098E07006758F
:1030ED006D04022C7A75BB170233F3900098E0B48F
:1030FD000102800302318C7E017F00E5BE12697AE8
:10310D00E5BD2FFF50010E8E588F599007E4E060FA
:10311D00199007E4E0149063F412008CE493FC74AE
:10312D000193FDEDC39FEC9E400280069007E4E005
:10313D0014F09007E4E0C394B3501DAE58AF59900E
:10314D0007E4E0049063F412008CE493FC740193A3
:10315D00FDEFC39DEE9C400280069007E4E004F075
:10316D009007E4E0FE9000BEE08E0088F0A4FFAE74
:10317D00F074648E048F05FF12696A8D6580037586
:10318D006500900099E07006756D05022C7A75BB8F
:10319D00160233F3900099E0B40102800302323538
:1031AD007E017F00E5BE12697AE5BD2FFF50010E4D
:1031BD008E588F599007E5E060199007E5E014905F
:1031CD00655E12008CE493FC740193FDEDC39FECDE
:1031DD009E400280069007E5E014F09007E5E0C3FD
:1031ED0094B3501DAE58AF599007E5E00490655E5D
:1031FD0012008CE493FC740193FDEFC39DEE9C4093
:10320D000280069007E5E004F09007E5E0FE9000EF
:10321D00C4E08E0088F0A4FFAEF074648E048F05B8
:10322D00FF12696A8D66800375660075BB1F0233D8
:10323D00F37E017F00E5BE12697AE5BD2FFF5001D7
:10324D000E8E588F59740912697A74E68E048F05A3
:10325D00FF12696A8D689000A0E07006756D070217
:10326D002C7A75BB150233F39000A0E07003023386
:10327D008F7E017F00E5BE12697AE5BD2FFF5001FB
:10328D000E8E588F5974041200398F679000A0E08C
:10329D00B401159000F4E08567F0A4FFAEF074075B
:1032AD00120039EF9007D9F09000A0E0B40215900C
:1032BD0000F4E08567F0A4FFAEF07407120039EF5B
:1032CD009007D8F09000A0E0B40302800302338D84
:1032DD009000E1E070389000F4E0601CE567C39465
:1032ED00195002D226E567D394644002C22690009D
:1032FD00C0E09007DCF08014E567C394195002D24A
:10330D0035E567D394324002C235C2268063900002
:10331D00C0E070349000F4E08567F0A4FFAEF07467
:10332D00FF8E048F05FF12696AED9007DCF0AE5039
:10333D00AF51741EBE0006D39F4002D226E55FD367
:10334D0094E54002C2268029E567C3940A500DAE6C
:10335D0050AF51741EBE0004D39F50028002D2267E
:10336D00E55FD394E54002C2269000C0E09007DCF3
:10337D00F09007DCE0C39405500674059007DCF06F
:10338D0080037567009000F7E07006756D08022CDC
:10339D007A75BB1480509000F7E060397E017F0094
:1033AD00E5BE12697AE5BD2FFF50010E8E588F597B
:1033BD00EFD39421EE940E40057569FF8015AE583C
:1033CD00AF59741012697A74E38E048F05FF126978
:1033DD006A8D69800375690090009BE0600575BB7F
:0633ED001A800375BB18F5
:10359F00022C83022E3D022FDE0230930230F802FE
:0B35AF0031A102323E0232750233A34C
:0533F300056DD2EC2283
:0969AC002582F5825002058322C8
:0F008C0025E050020583258250020583F582226C
:10694900EF2F500205832582F582E5833E2EF583DC
:01695900221B
:1069BE00CFC39FFF50011E22C3EF9DFFEE9CFE2210
:0869CE000806B60002180622BB
:0D698800A3E004F07006120049E004F022C4
:0E003900048007C3CE13CECF13CFD5E0F6223E
:10686800BC000FBE0008ED8FF084FFADF022E4FEFF
:10687800FF22BE000DEF60FE54F0606F20E70302B8
:10688800691EEAC0E0EBC0E078017A0075F001EE1D
:1068980020E710EF25E0FFEE33FE0AC5F023C5F030
:1068A80030E7F0EA5407F9096A7A007B00600108CA
:1068B800C3EC9E40167004ED9F4010ED9FFDEC9ECA
:1068C800FCE5F0CA4ACA03F5F08005E5F003F5F0E7
:1068D800C3EE13FEEF13FFD9D77908CACBCAD8D0B5
:1068E800EAFEEBFFD0E0FBD0E0FA22EC8FF084FC6C
:1068F800ED54F045F0C48FF084FEEDC454F045F03B
:10690800C48FF084FDEEC4FE54F02DFFEE540F3C0E
:10691800FEADF07C0022790078008FF0EC7E082034
:10692800E70DC3CD33CD33C933C9C833C8DEF084CE
:1069380049F9E5F08FF0BE00E6FD7C00E9FFE8FECE
:01694800222C
:0E697A00F88FF0A4FFE5F0CE88F0A42EFE22E8
:10000300EF8DF0A4F9A8F0EF8CF0A428F8EE8DF0B2
:06001300A428FEE9FF2213
:10695A00600D782B026964007830D8FED5E0F82201
:10696A00EEC0E07E00126868EFFDEEFCD0E0FE2289
:0C699500EEC0E07E00126868D0E0FE2238
:03001B0002001EC2
:0300530002005652
:03009B00020071EF
:030000000269B5DD
:0969B50075817375D000024002E7
:0B69A100E5822FF582E5833EF583229E
:0A0049000582D5820215831582227C
:10001E00C0E0C0F0C083C082C0D075D000123FA631
:0B002E00D0D0D082D083D0F0D0E032E0
:10005600C0E0C0F0C083C082C0D075D000123FA9F6
:10006600D0D0D082D083D0F0D0E032C0E0C0F0C093
:1000760083C082C0D075D000123FCBD0D0D082D002
:0600860083D0F0D0E0324F
:00000001FF
